:10000000A2C20000D1C20000CFC20000CDC20000D9
:10001000CBC20000C9C20000C7C20000C5C20000B8
:10002000C3C20000C1C20000BFC20000BDC20000C8
:10003000BBC20000B9C20000B7C20000B5C20000D8
:10004000B3C200000C94C809AFC20000ADC20000EA
:100050000C942D0DA9C20000A7C200000C94E30C63
:10006000A3C200000C94BB0B0C94920B9DC2000029
:100070009BC2000099C2000097C2000095C2000018
:100080000C949B0991C200008FC200008DC2000039
:100090008BC2000089C2000087C2000085C2000038
:1000A00083C2000081C200000C946E097DC2000072
:1000B0007BC2000079C2000077C200000C944109A5
:1000C00073C2000071C200006FC200006DC2000068
:1000D0006BC2000069C2000067C2000065C2000078
:1000E00063C200001A0B1D0B0C0B100B160B540BEC
:1000F000210B250B2B0B2F0B330B390B3D0B410B1E
:10010000540B470B4B0B4F0BB412C112CA12D31234
:10011000E012E91285168516851685168516F612E3
:100120000313101385161D1326132F133C134513A9
:100130004E13571360136913851672137B138413C0
:100140008516851685168D1396139F1385168516AD
:10015000A813B513851685168516C213CF13DC13A5
:100160008516E913F213FB138516851685160414FC
:100170000D1416148516231430143D148516851697
:1001800085164A1457146414851671147E148B1442
:100190008516851685169814A514B2148516BF14F5
:1001A000C814D114851685168516851685168516EC
:1001B0008516851685168516851685168516851667
:1001C0008516851685168516851685168516851657
:1001D0008516F514FE140715851610151915221528
:1001E0008516851685162B15381545158516521555
:1001F0005F156C1585168516851679158615931568
:100200008516A015A915B215851685168516BB1578
:10021000C415CD1585168516851685168516851681
:1002200085168516851685168516DA14E314EC14E2
:1002300085168516851685168516851685168516E6
:1002400085168516851685168516851685168516D6
:1002500085168516851685168516851685168516C6
:1002600085168516851685168516851685168516B6
:1002700085168516851685168516851685168516A6
:100280008516851685168516851685168516851696
:1002900085168516851685168516D615DF15EC1577
:1002A0008516F91502160F168516851685161C1665
:1002B0002516321685163F164816551685168516CC
:1002C000851662166B16781608180D1812181C1869
:1002D00026189F183018381840184A1854185E18F5
:1002E0006D1877189F1881188B1895184E414E4934
:1002F0004E495459494E46CDCCCC3D0AD7233C17E4
:10030000B7D13877CC2B329595E6241FB14F0A0030
:100310000020410000C84200401C4620BCBE4CCA20
:100320001B0E5AAEC59D7400407A10F35A00A0729D
:100330004E18090010A5D4E80000E8764817000020
:10034000E40B54020000CA9A3B000000E1F50500EE
:100350000080969800000040420F000000A0860137
:10036000000000102700000000E803000000006407
:1003700000000000000A0000000000010000000072
:10038000002C76D888DC674F0823DFC1DFAE59E147
:10039000B1B796E5E3E453C63AE651997696E8E6B6
:1003A000C28426EB898C9B62ED407C6FFCEFBC9C89
:1003B0009F40F2BAA56FA5F490055A2AF75C936B9B
:1003C0006CF9676DC11BFCE0E40D47FEF520E6B556
:1003D00000D0ED902E0300943577050080841E0830
:1003E0000000204E0A000000C80C333333330F984E
:1003F0006E12831141EF8D2114893BE65516CFFE15
:10040000E6DB18D1844B381BF77C1D901DA4BBE4A0
:1004100024203284725E228100C9F124ECA1E53DE2
:100420002700002100240027002A002D003000337F
:100430000001010000040107010A0101021020204F
:100440000808102040102040800201020108040228
:10045000010102040810204080804020100804029E
:1004600001800402018040201008040201080402F7
:1004700001010204081020408001020408102040FD
:100480008005050505070508080808020202020A9A
:100490000A08080404040401010101010101010327
:1004A00003030303030303040707070C0C0C0C0CE2
:1004B0000C0C0C0202020206060606060606060BD5
:1004C0000B0B0B0B0B0B0B00000A0B02090C0D0E98
:1004D0000807030401000000000000000000000005
:1004E000000000000000000000000000000000000C
:1004F00000000012111000000000000000000000C9
:1005000000000000000000000000000000000022C9
:1005100000250028002B002E0031003400020100CD
:1005200000050108010B010000200023002600291E
:10053000002C002F00320000010000030106010919
:100540000100D945D44511241FBECFEFD1E2DEBF53
:10055000CDBF00E00CBF17E0A0E0B2E0EEEAFFE99B
:1005600000E00BBF02C007900D92AE32B107D9F781
:100570002CE0AEE2B7E001C01D92A93DB207E1F761
:1005800012E0C2EAD2E000E006C021970109802F04
:10059000FE010E94BA4EC13AD10780E00807A9F7D0
:1005A0000E94E73B0C94C64F2BCDCF92DF92EF9287
:1005B000FF92CF93DF93EC01603282E078070CF07A
:1005C0003DC077FD06C0653B71052CF064EB70E023
:1005D00002C060E070E0898128E830E06901C81A53
:1005E000D10887FDD394CC0CDD1CCC0CDD1C0D2C6C
:1005F000000CEE08FF088A8128E532E0281B31094B
:1006000087FD3395220F331F220F331FC901330F8C
:10061000AA0BBB0B9C01AD012C193D094E095F09CA
:10062000DB010E947D4D24EB30E040E050E00E9471
:10063000574DC20ED31EE41EF51EB60188818033CD
:1006400080F5998148E850E0491B510997FD539581
:10065000440F551F440F551F6417750784F09A8186
:1006600028E532E0291B310997FD3395220F331F0E
:10067000220F331FAB01261737070CF4A901425094
:100680005109440F551F2FB7F89490E0FC01EE0F6D
:10069000FF1F8E0F9F1FFC01EE5CF34F52834183BF
:1006A0002FBFDF91CF91FF90EF90DF90CF90089513
:1006B000662319F081EE93E002C08AED93E00C947A
:1006C00020370C9413470C9413470C9413470C9445
:1006D00013470C9413470C9413470C9413470C9432
:1006E00013470C9413470C9413470C9413470C9422
:1006F00013470C9413470C9413470C9413470C9412
:1007000013470C9413470C9413470F931F93CF93E5
:10071000DF93FB0102A913A9C68DD78D0E94AC18E7
:10072000A801BE010E94CE2880E090E0DF91CF9129
:100730001F910F9108950F931F93CF93DF93FB01A8
:10074000C2A1D3A1068D178D8091810B9091820B50
:10075000892B41F481E090E00E947E469093820BC9
:100760008093810B0430110539F00530110541F4F7
:10077000BE0186EC9CE003C0BE0183EC9CE015DF6B
:1007800080E090E0DF91CF911F910F910895EF925B
:10079000FF920F931F93CF93DF93FB01E2A8F3A87F
:1007A00002A113A1C68DD78D0E94AC189701A80194
:1007B000BE010E94C41780E090E0DF91CF911F91AD
:1007C0000F91FF90EF9008956F927F928F929F927A
:1007D000AF92BF92CF92DF92EF92FF920F931F934F
:1007E000CF93DF93FB01E2A8F3A886A497A4A0A867
:1007F000B1A8C6A0D7A062A073A0068D178D0E94D5
:10080000AC18EC019701A301B8010E94C417C501FF
:10081000B4010E949F0C9701A601B801CE010E946D
:10082000C41780E090E0DF91CF911F910F91FF906E
:10083000EF90DF90CF90BF90AF909F908F907F9080
:100840006F9008951F93CF93DF931F92CDB7DEB7BC
:10085000FB0162A9168D69830E94AC186981812F02
:100860000E94580C80E090E00F90DF91CF911F9193
:100870000895CF93DF93FB01C68DD78D0E94F219A7
:10088000BE010E94B01980E090E0DF91CF91089501
:10089000EF92FF920F931F93CF93DF9300D01F929D
:1008A000CDB7DEB7FB0122A133A144A155A1068D2E
:1008B000178D29833A834B835C830E94F2197C0154
:1008C000FC018281938129813A814B815C818F3047
:1008D000F7E29F072CF40196F7019383828303C00C
:1008E000F70113821282B801C70129833A834B832F
:1008F0005C830E94CB1829813A814B815C818823DB
:10090000A1F0F801EE0FFF1FEE0FFF1FEE5CF84F96
:100910002083318342835383B801C7010E94611948
:10092000B801C7010E94B01904C089E894E00E9490
:1009300020370E94A2280E94722880E090E00F9049
:100940000F900F900F90DF91CF911F910F91FF901B
:10095000EF9008958F929F92AF92BF92CF92DF92C5
:10096000EF92FF920F931F930E94592862E070E06C
:100970000E94A131892BD1F40E94592821E02F93A4
:100980001F921F921F921F92812C912CA12CB12C8F
:10099000C12CD12C760197018601B701A6010E94D6
:1009A000201B0F900F900F900F900F9080E090E021
:1009B0001F910F91FF90EF90DF90CF90BF90AF907D
:1009C0009F908F9008958F929F92AF92BF92CF92F7
:1009D000DF92EF92FF920F931F930E94592861E0DC
:1009E00070E00E94A131892BD1F40E9459281F92F6
:1009F00021E02F931F921F921F92812C912CA12CEA
:100A0000B12CC12CD12C760197018601B701A6012A
:100A10000E94201B0F900F900F900F900F9080E07E
:100A200090E01F910F91FF90EF90DF90CF90BF90DB
:100A3000AF909F908F9008958F929F92AF92BF92A8
:100A4000CF92DF92EF92FF920F931F930E9459284B
:100A500060E070E00E94A131892BD1F40E945928F6
:100A60001F921F9221E02F931F921F92812C912C95
:100A7000A12CB12CC12CD12C760197018601B70194
:100A8000A6010E94201B0F900F900F900F900F90C7
:100A900080E090E01F910F91FF90EF90DF90CF905A
:100AA000BF90AF909F908F9008958F929F92AF923A
:100AB000BF92CF92DF92EF92FF920F931F930E940B
:100AC000592821E02F931F921F921F921F92812C71
:100AD000912CA12CB12CC12CD12C7601970186012F
:100AE000B701A6010E94201B0F900F900F900F904E
:100AF0000F9080E090E01F910F91FF90EF90DF90BA
:100B0000CF90BF90AF909F908F9008958F929F92BB
:100B1000AF92BF92CF92DF92EF92FF920F931F930B
:100B20000E9459281F9221E02F931F921F921F921B
:100B3000812C912CA12CB12CC12CD12C76019701A8
:100B40008601B701A6010E94201B0F900F900F9005
:100B50000F900F9080E090E01F910F91FF90EF9029
:100B6000DF90CF90BF90AF909F908F9008958F921D
:100B70009F92AF92BF92CF92DF92EF92FF920F932C
:100B80001F930E9459281F921F9221E02F931F92BA
:100B90001F92812C912CA12CB12CC12CD12C76012F
:100BA00097018601B701A6010E94201B0F900F90AC
:100BB0000F900F900F9080E090E01F910F91FF90A9
:100BC000EF90DF90CF90BF90AF909F908F9008955F
:100BD000CF92DF92EF92FF920F931F93CF93DF9309
:100BE0006C018B017A01EC01CD58D44F888187FFCD
:100BF00004C0FB011182108224C08CE08C9D900106
:100C00008D9D300D11248881A901480F511D87FD4C
:100C10005A958091C20C90E04817590794F4888146
:100C2000A901480F511D87FD5A95CA01FA01EE0F1F
:100C3000FF1F8E0F9F1FFC01EE5CF34F808186FD2E
:100C400019C088818F5F88838CE08C9D90018D9D79
:100C5000300D11248881A901480F511D87FD5A9537
:100C60008091C20C90E048175907B4F488818C3009
:100C70003CF112C08881280F311D87FD3A95F9019A
:100C8000EE0FFF1F2E0F3F1FF901EE5CF34F808127
:100C900060E08F73CED5D5CFF80180819181049625
:100CA00080349C4918F480E49CE904C0F8018081F8
:100CB00091810496F701918380838FEF888344C0EC
:100CC000F801408151818881B901680F711D87FD4C
:100CD0007A95CB01FB01EE0FFF1F8E0F9F1FFC01CA
:100CE000EE5CF34F81819281840F951FF701918310
:100CF00080838881A901480F511D87FD5A95CA013B
:100D0000FA01EE0FFF1F8E0F9F1FFC01EE5CF34FE9
:100D1000808186FF19C08881280F311D87FD3A9593
:100D2000F901EE0FFF1F2E0F3F1FF901EE5CF34F8D
:100D3000808161E08F73DF91CF911F910F91FF90C0
:100D4000EF90DF90CF9075C5DF91CF911F910F91FC
:100D5000FF90EF90DF90CF90089508950895089543
:100D6000089508950895089508950895089508959B
:100D70000895089508950895089508950895EF92A7
:100D8000FF920F931F93CF93DF93CDB7DEB72E97CC
:100D90000FB6F894DEBF0FBECDBF8C0162ED73E0DD
:100DA0000E9418396BEA74E0C8010E94DA38609139
:100DB000B60A7091B70A8091B80A9091B90A2AE0F0
:100DC000AE014F5F5F4F7A010E94E247F701019049
:100DD0000020E9F73197AF014E195F09B701C8014B
:100DE0000E947D3860ED73E0C8010E94DA38C801C6
:100DF0002E960FB6F894DEBF0FBECDBFDF91CF9118
:100E00001F910F91FF90EF9008958BEA94E00E945C
:100E100020376091B60A7091B70A8091B80A909114
:100E2000B90A0E946C3780ED93E00C9420370F9341
:100E30001F93CF93DF93EC018EEA94E00E9420375A
:100E400082EB94E00E9420370BE71BE0F801608101
:100E5000CE012EDC86EB94E00E942037F801618100
:100E6000CE0126DC8AEB94E00E942037F8016281F3
:100E7000CE011EDC8EEB94E00E942037F8016381E6
:100E8000CE0116DC82EC94E00E942037F8016481E8
:100E9000CE010EDC86EC94E00E942037F8016581DB
:100EA000CE0106DCCE01DF91CF911F910F91ADCF26
:100EB000CF92DF92EF92FF92CF93DF93EC01888184
:100EC0009981AA81BB81181619061A061B0644F0DF
:100ED00081E090E0A0E0B0E088839983AA83BB839F
:100EE0008C819D81AE81BF81181619061A061B06DA
:100EF00044F081E090E0A0E0B0E08C839D83AE837D
:100F0000BF8388859985AA85BB85181619061A0698
:100F10001B0644F081E090E0A0E0B0E0888799876C
:100F2000AA87BB878AEC94E00E9420378BED94E07F
:100F30000E9420376091BA0A7091BB0A8091BC0A66
:100F40009091BD0A0E942B4C6B017C0168817981D4
:100F50008A819B810E942B4C9B01AC01C701B60189
:100F60000E94194E42E00E9493378BEE94E00E945B
:100F700020376091BE0A7091BF0A8091C00A90919B
:100F8000C10A0E942B4C6B017C016C817D818E819A
:100F90009F810E942B4C9B01AC01C701B6010E94AE
:100FA000194E42E00E9493378BEF94E00E94203765
:100FB0006091C20A7091C30A8091C40A9091C50AD7
:100FC0000E942B4C6B017C01688579858A859B8505
:100FD0000E942B4C9B01AC01C701B6010E94194E27
:100FE00042E00E949337CE01DF91CF91FF90EF90C6
:100FF000DF90CF900ACF8091790B90917A0B892B5B
:1010000091F58DE090E00E947E46FC0114861092DE
:10101000BA0A1092BB0A1092BC0A1092BD0A109232
:10102000BE0A1092BF0A1092C00A1092C10A109212
:10103000C20A1092C30A1092C40A1092C50A1092F2
:10104000780B1092770B1092B60A1092B70A109292
:10105000B80A1092B90A1092310710923007909393
:101060007A0B8093790B8091790B90917A0B08958C
:10107000CF93DF93EB0120E030E040E85FE36A814B
:101080007B818C819D810E94254C811111C08EEC49
:1010900094E00E9420370E945928FC01E25BFF4F38
:1010A000108211821282138282589E4F0E946738EA
:1010B00020E030E040E85FE36E817F81888599859C
:1010C0000E94254C811111C08EED94E00E942037C2
:1010D0000E945928FC01E853FF4F108211821282AE
:1010E000138286569E4F0E94673820E030E040E829
:1010F0005FE36A857B858C859D850E94254C8111E7
:1011000011C08EEE94E00E9420370E945928FC0105
:10111000EE5BFE4F10821182128213828A549E4F20
:101120000E94673868DF71DE80E090E0DF91CF9148
:1011300008958EEF94E00E9420378DE093E00E94A6
:10114000203759DF62DE80E090E0089554DFB0DEA2
:1011500080E090E008950F931F93CF93DF930E9458
:10116000F2198C01C0E0D0E0BE01C8010E94CB188A
:10117000882321F0BE01C8010E94B0192196C13E0A
:10118000D10591F783E095E00E94203734DF3DDE02
:1011900080E090E0DF91CF911F910F9108952BDFB8
:1011A000FC01148680E090E00895CF93DF9385E4FE
:1011B00018D3EC0120DF91E0CD2B09F490E090935F
:1011C0007B0B84E40ED3EC0116DF91E0CD2B09F408
:1011D00090E090937C0B83E404D3EC010CDF91E06E
:1011E000CD2B09F490E090937D0B82E4FAD2EC01D0
:1011F00002DF91E0CD2B09F490E090937E0B81E427
:10120000F0D2EC01F8DE91E0CD2B09F490E0909360
:101210007F0B80E4E6D2EC01EEDE91E0CD2B09F409
:1012200090E09093800BDF91CF91089587E095E057
:101230000E942037E0DEB9DFDEDEF9DD0E94AC1867
:1012400040E050E068E070E00E94CE280E94AC18B8
:1012500040E050E069E070E00E94CE280E94AC18A7
:1012600040E050E06AE070E00E94CE280E94AC1896
:1012700040E050E06DE070E00E94CE2880E090E019
:1012800008951F920F920FB60F9211240BB60F9272
:101290002F933F934F935F936F937F938F939F937E
:1012A000AF93BF93EF93FF9348E251E064E271E0A4
:1012B00080E090E08DDCFF91EF91BF91AF919F9125
:1012C0008F917F916F915F914F913F912F910F90EF
:1012D0000BBE0F900FBE0F901F9018951F920F928C
:1012E0000FB60F9211240BB60F922F933F934F938B
:1012F0005F936F937F938F939F93AF93BF93EF937E
:10130000FF9348EA50E064EA70E083E090E060DC3C
:10131000FF91EF91BF91AF919F918F917F916F91CD
:101320005F914F913F912F910F900BBE0F900FBE89
:101330000F901F9018951F920F920FB60F921124C5
:101340000BB60F922F933F934F935F936F937F93BF
:101350008F939F93AF93BF93EF93FF9348E950E030
:1013600064E970E082E090E033DCFF91EF91BF919F
:10137000AF919F918F917F916F915F914F913F912D
:101380002F910F900BBE0F900FBE0F901F901895CE
:101390001F920F920FB60F9211240BB60F922F933C
:1013A0003F934F935F936F937F938F939F93AF93ED
:1013B000BF93EF93FF9348E850E064E870E081E06A
:1013C00090E006DCFF91EF91BF91AF919F918F91DB
:1013D0007F916F915F914F913F912F910F900BBE35
:1013E0000F900FBE0F901F901895089580E090E029
:1013F0000895FC01538D448D252F30E0842F90E01B
:10140000821B930B541710F0CF96089501970895FF
:10141000FC01918D828D981761F0828DDF01A80FFC
:10142000B11D5D968C91928D9F5F9F73928F90E01E
:1014300008958FEF9FEF0895FC01918D828D98178D
:1014400031F0828DE80FF11D858D90E008958FEFCA
:101450009FEF0895FC01918D228D892F90E0805C93
:101460009F4F821B91098F739927089585E99BE00F
:10147000F1DF21E0892B09F420E0822F0895FC019F
:10148000848DDF01A80FB11DA35ABF4F2C91848D0D
:1014900090E001968F739927848FA689B7892C9342
:1014A000A089B1898C9180648C93938D848D9813DD
:1014B00006C00288F389E02D80818F7D80830895A6
:1014C000EF92FF920F931F93CF93DF93EC0181E094
:1014D000888F9B8D8C8D981305C0E889F989808150
:1014E00085FD23C0F62E0B8D10E00F5F1F4F0F738D
:1014F0001127E02E8C8DE8120BC00FB607FCFACF37
:10150000E889F989808185FFF5CFCE01B8DFF2CF78
:101510008B8DFE01E80FF11DE35AFF4FF0820B8F18
:10152000EA89FB898081806207C0EE89FF89608338
:10153000E889F98980818064808381E090E0DF918F
:10154000CF911F910F91FF90EF900895CF93DF936C
:10155000EC01888D8823C1F0EA89FB89808185FDB3
:1015600005C0A889B9898C9186FD0EC00FB607FC0D
:10157000F5CF808185FFF2CFA889B9898C9185FF4D
:10158000EDCFCE017CDFE8CFDF91CF91089580E0F1
:1015900090E0892B19F06ADF811125C080E090E08E
:1015A000892B41F080E090E0892B21F00E9400001F
:1015B00081111CC080E090E0892B41F080E090E038
:1015C000892B21F00E940000811113C080E090E07F
:1015D000892BA1F080E090E0892B81F00E9400002F
:1015E00081110AC008950E940000D8CF0E94000017
:1015F000E1CF0E940000EACF0C940000089590E033
:10160000FC013197E231F10508F04EC08827EE5811
:10161000FF4F8F4F0C94BA4E809180008F7703C09C
:10162000809180008F7D809380000895809180005C
:10163000877FF9CF84B58F7702C084B58F7D84BD55
:1016400008958091B0008F7703C08091B0008F7DA6
:101650008093B0000895809190008F7707C08091AB
:1016600090008F7D03C080919000877F80939000D1
:1016700008958091A0008F7707C08091A0008F7D92
:1016800003C08091A000877F8093A000089580917F
:1016900020018F7707C0809120018F7D03C080914A
:1016A0002001877F8093200108953FB7F8948091AF
:1016B000880B9091890BA0918A0BB0918B0B26B56A
:1016C000A89B05C02F3F19F00196A11DB11D3FBF7A
:1016D000BA2FA92F982F8827820F911DA11DB11D08
:1016E000BC01CD0142E0660F771F881F991F4A9504
:1016F000D1F70895EBE0F1E08081877F8083089542
:10170000EBE0F1E080818860808308958E980895F1
:101710008E9A089514980895149A089588980895B3
:10172000889A08951F920F920FB60F9211240BB64C
:101730000F922F933F934F935F936F937F938F936A
:101740009F93AF93BF93EF93FF9385E99BE097DE61
:10175000FF91EF91BF91AF919F918F917F916F9189
:101760005F914F913F912F910F900BBE0F900FBE45
:101770000F901F9018951F920F920FB60F92112481
:101780000BB60F922F938F939F93EF93FF93E0915C
:10179000A50BF091A60B8081E091AB0BF091AC0B07
:1017A00082FD12C090818091AE0B8F5F8F7320916C
:1017B000AF0B821751F0E091AE0BF0E0EB56F44F17
:1017C000958F8093AE0B01C08081FF91EF919F9127
:1017D0008F912F910F900BBE0F900FBE0F901F9007
:1017E0001895CF93DF93282F30E0F901E953FB4F91
:1017F0008491F901E55CFB4FD491F901EF57FB4F60
:10180000C491CC2389F08111FADEEC2FF0E0EE0FC9
:10181000FF1FE95DFA4FA591B491EC91ED2381E0B2
:1018200090E021F480E002C080E090E0DF91CF9171
:1018300008951F93CF93DF93282F30E0F901E953E8
:10184000FB4F8491F901E55CFB4FD491F901EF570F
:10185000FB4FC491CC23C1F0162F8111D0DEEC2FA9
:10186000F0E0EE0FFF1FE35FFA4FA591B4918FB741
:10187000F894111105C09C91ED2FE095E92302C069
:10188000EC91ED2BEC938FBFDF91CF911F910895D9
:1018900060E0FC018385CDCF60E0FC018581C9CF8C
:1018A00061E0FC018385C5CF61E0FC018581C1CF8A
:1018B000CF93DF9390E0FC01E55CFB4F2491FC01AA
:1018C000EF57FB4F8491882361F190E0880F991FB7
:1018D000FC01EF5DFB4FC591D491FC01E35FFA4F32
:1018E000A591B491611109C09FB7F89488812095A2
:1018F00082238883EC912E230BC0623061F49FB762
:10190000F8943881822F809583238883EC912E2B45
:101910002C939FBF06C08FB7F894E8812E2B2883A5
:101920008FBFDF91CF9108958230910538F0880FF5
:10193000991F880F991F05970197F1F708958F92C6
:101940009F92AF92BF92CF92DF92EF92FF926B0184
:101950007C01ABDE4B015C01C114D104E104F10454
:10196000E9F0A3DEDC01CB0188199909AA09BB09BA
:10197000883E9340A105B10578F321E0C21AD10851
:10198000E108F10888EE880E83E0981EA11CB11CC6
:10199000C114D104E104F10421F7DECFFF90EF90F0
:1019A000DF90CF90BF90AF909F908F9008952FB70A
:1019B000F8946091840B7091850B8091860B9091C7
:1019C000870B2FBF08951F920F920FB60F9211240D
:1019D0002F933F938F939F93AF93BF938091840BEB
:1019E0009091850BA091860BB091870B3091830B62
:1019F00023E0230F2D3720F40196A11DB11D05C052
:101A000026E8230F0296A11DB11D2093830B80931E
:101A1000840B9093850BA093860BB093870B8091DA
:101A2000880B9091890BA0918A0BB0918B0B01963A
:101A3000A11DB11D8093880B9093890BA0938A0BF5
:101A4000B0938B0BBF91AF919F918F913F912F914D
:101A50000F900FBE0F901F9018951F920F920FB608
:101A60000F9211240BB60F922F933F934F935F93D6
:101A70006F937F938F939F93AF93BF93EF93FF9356
:101A8000E0912E07F0912F071995FF91EF91BF91EB
:101A9000AF919F918F917F916F915F914F913F9106
:101AA0002F910F900BBE0F900FBE0F901F901895A7
:101AB000CF93DF93FC01A489B589C08DD18D208996
:101AC000318942895389A03187E2B80759F01A1643
:101AD0001B0644F40E947D4D20E137E240E050E0D7
:101AE0000E94574DDE010E947D4DDF91CF910895F8
:101AF000FC0181E090E0938F828F11821082158229
:101B00001482108A118A128A138A178A168A80E12F
:101B100097E2958B848B128610861486158616861E
:101B2000178608958EBD00000DB407FEFDCF8EB55B
:101B30000895CF92DF92EF92FF920F931F93CF936E
:101B4000DF93EC0160E086E174DE8A8D9B8D24E0FA
:101B5000880F991F2A95E1F78F60E4DF83E290E018
:101B60000197F1F704E010E0C12CD12C7601FE2C96
:101B7000ED2CDC2CCC2481E0D5DFC82A01501109E2
:101B8000B1F761E086E155DEC88AD98AEA8AFB8A24
:101B9000DF91CF911F910F91FF90EF90DF90CF9049
:101BA0000895CF93DF93EC01FC01E759FF4F1082BA
:101BB000379781E0808360E08D813BDE8F85988957
:101BC000892B29F060E08B85DF91CF9132CEDF91B8
:101BD000CF910895CF93DF93EC018B8902DE2E899C
:101BE00030E08217930711F48F8901C080E0DF9104
:101BF000CF910895CF93DF93EC018989F2DD2E898F
:101C000030E08217930711F48F8901C080E0DF91E3
:101C1000CF910895CF93DF93EC018DA5882311F028
:101C200061E001C060E08F8104DE8EA5882329F089
:101C30008FA5882311F061E001C060E08D85DF9100
:101C4000CF91F7CDCF93DF93EC018DA5882311F0D1
:101C500060E001C061E08F81ECDD8EA5882329F072
:101C60008FA5882311F060E001C061E08D85DF91D0
:101C7000CF91DFCDCF93DF93EC0161E08985D9DD92
:101C80008EA5882319F061E08F85D3DDC959DF4F18
:101C90001882DF91CF910895CF93DF93EC0160E03C
:101CA0008985C7DD8EA5882319F060E08F85C1DDA9
:101CB000C959DF4F81E08883DF91CF910895CF929A
:101CC000DF92EF92FF920F931F93CF93DF93FC016C
:101CD00042AF53AF64AF75AFDC01DE964D935D93B9
:101CE0006D937C93139714960D931D932D933C93B2
:101CF0001397EC01CA5BDF4FE88284A9882351F077
:101D000084A581114BC037FF05C01D921D921D9205
:101D10001C92139745A956A967A970AD141615060C
:101D20001606170634F581AD882319F10D911D9122
:101D30002D913C9113976801790137FF07C0CC249E
:101D4000DD247601C01AD10AE20AF30A4C155D05BA
:101D50006E057F0574F437FF07C070956095509548
:101D600041955F4F6F4F7F4F4D935D936D937C9384
:101D70001397DF01A15BBF4F1D921D921D921C9214
:101D80001397E15AFF4F81E08083DF91CF911F913C
:101D90000F91FF90EF90DF90CF90089510161106ED
:101DA000120613060CF4B1CFB5CF0F931F93CF9348
:101DB000DF938C01D62FFC018589811109C0C801F0
:101DC00019DFC82FC80106DFD11108C08C2F06C04B
:101DD000C80100DFC82FC8010DDFF6CFDF91CF911A
:101DE0001F910F910895CF93DF93EC01FC01E75908
:101DF000FF4F81E0808339978081B297882341F03B
:101E000080819181A281B3810196A11DB11D07C07E
:101E100080819181A281B3810197A109B109808359
:101E20009183A283B383FE01E459FF4F2081318166
:101E3000DE01A659BF4FC9019595879520FD03C0C6
:101E4000ED91FC910DC0FE01E80FF91F0190F081AA
:101E5000E02D2D913C91E20FF31F0190F081E02DD8
:101E60008C0F9D1F19958F859889892B11F1FE0183
:101E7000E059FF4F20813181DE01A259BF4FC901D6
:101E80009595879520FD03C0ED91FC910DC0FE0155
:101E9000E80FF91F0190F081E02D2D913C91E20FA8
:101EA000F31F0190F081E02D8C0F9D1FDF91CF91EA
:101EB0001994DF91CF9108958F929F92AF92BF9224
:101EC000CF92DF92EF92FF920F931F93CF93DF9306
:101ED000EC01FC01E15BFF4F6081718182819381A4
:101EE0000E94294C6B017C0168A979A98AA99BA948
:101EF0000E942B4C9B01AC0160E074E284E799E402
:101F00000E94194E4B015C01FE01E55AFF4F6081B2
:101F10007181828193810E94294C9B01AC01C50192
:101F2000B4010E94194E4B015C018E010D5A1F4FE6
:101F300020E030E040E05FE30E948A4C9B01AC016E
:101F4000C701B6010E94B54D0E94864EF80160831C
:101F5000718382839383C95ADF4FA5019401C7011E
:101F6000B6010E94B54D0E94864E688379838A83AC
:101F70009B83DF91CF911F910F91FF90EF90DF90A6
:101F8000CF90BF90AF909F908F9008950F931F9325
:101F9000CF93DF93FC01E759FF4F20812223B9F053
:101FA0007A97008111812281338138964081518155
:101FB00062817381041715072607370710F1EC01BA
:101FC000F0DDCE01DF91CF911F910F9175CFFC0114
:101FD000E15AFF4F20812223A1F0709700811181E7
:101FE000228133813496408151816281738104174B
:101FF00015072607370728F0DF91CF911F910F9122
:10200000F2CEDF91CF911F910F9108952F923F92C1
:102010004F925F926F927F928F929F92AF92BF92F8
:10202000CF92DF92EF92FF920F931F93CF93DF93A4
:10203000CDB7DEB762970FB6F894DEBF0FBECDBF47
:102040008C017C0126E4E20EF11CD7018C919801F1
:10205000205A3F4FF801EF59FF4F6F01A801425C32
:102060005F4F4A0114971D01882341F0F80184A5B0
:10207000D9018C9381E0F60180832FC0DA014D9164
:102080005D916D917C91F10180819181A281B381FB
:10209000BB24B394481759076A077B070CF0B12C8F
:1020A000F901B08277FF07C0709560955095419512
:1020B0005F4F6F4F7F4FB7FF07C0B095A0959095CA
:1020C00081959F4FAF4FBF4F21E0481759076A07CF
:1020D0007B070CF420E0D6012C93F4014081518160
:1020E00062817381411551056105710559F4F8014B
:1020F000848D958DA68DB78DE55AFF4F8083918392
:10210000A283B383F10180819181A281B381F8011F
:1021100042AC53AC64AC75AC9801215A3F4F5901A5
:10212000481659066A067B0634F4481759076A07A9
:102130007B077CF00AC084159505A605B7052CF42D
:1021400084179507A607B70724F0D7018C91882339
:10215000D9F0F50180818823B9F0D7018C918111E4
:1021600005C0F701808181110FC006C060E0C80181
:102170001CDE8111F6CF17C0D6016C9181E0682773
:10218000C80113DE882379F0D5011C9260E0C801F4
:102190000CDE882309F4C4C1F801FE961082118276
:1021A00012821382BDC1D80194962D913D914D911B
:1021B0005C91979729833A834B835C8358962D9142
:1021C0003D914D915C915B972D833E834F83588762
:1021D0005C962D913D914D915C915F9729873A874F
:1021E0004B875C87F10180819181A281B381F801E5
:1021F000FE96C080D180E280F380F80142AD53ADFD
:1022000064AD75ADED59FF4F1082319610823801E3
:10221000F5E66F0E711CF301108298012A593F4FA9
:10222000F9011082329610824C015D01841A950AE0
:10223000A60AB70AB7FE08C0B094A0949094809400
:10224000811C911CA11CB11C481759076A077B0708
:102250002CF4C41AD50AE60AF70A04C0C81AD90A27
:10226000EA0AFB0AD501C401B595A795979587950C
:102270008D879E87AF87B88BD801A859BF4F1D01A6
:10228000F7FC05C08C149D04AE04BF044CF4F801A7
:1022900000A0F1A1E02DFA8BE98B81E0D9011BC0F0
:1022A0002D853E854F8558892C153D054E055F05CA
:1022B00008F454C089819A81AB81BC818C159D053D
:1022C000AE05BF0564F42D813E812F5F3F4F3A8BF1
:1022D000298B81E0D3018C93F10180839EC0C701DB
:1022E000B6010E942B4C2B013C0169817A818B81C4
:1022F0009C810E942B4C9B01AC01C301B2010E9446
:10230000194E2B013C016D817E818F819885298535
:102310003A854B855C85621B730B840B950B0E9481
:102320002B4C9B01AC01C301B2010E948A4C2B01D2
:102330003C0169857A858B859C850E942B4C9B018D
:10234000AC01C301B2010E94B54D0E94814E7A8B4F
:10235000698B81E0F801ED59FF4F5CC0D501C401E4
:1023600029813A814B815C81821B930BA40BB50BB5
:10237000C816D906EA06FB065CF42D813E812E5F65
:102380003F4F3A8B298B81E0F801EB59FF4F42C058
:10239000C501B4016C197D098E099F090E942B4C5F
:1023A0002B013C0169817A818B819C810E942B4C9D
:1023B0009B01AC01C301B2010E94194E2B013C01EB
:1023C0006D817E818F81988529853A854B855C85D5
:1023D000621B730B840B950B0E942B4C9B01AC0171
:1023E000C301B2010E948A4C2B013C0169857A85A8
:1023F0008B859C850E942B4C9B01AC01C301B201D3
:102400000E94B54D0E94814E7A8B698B81E0F80164
:10241000EC59FF4F8083D1018C93F801848188238C
:10242000A9F0C5DAD80112964D905C901397052C4F
:10243000000C66087708DC01CB0184199509A60910
:10244000B709893E9340A105B10568F4F801E55A42
:10245000FF4F29893A89C901A0E0B0E080839183C8
:10246000A283B38393CEA3DAD80113967C936E93A1
:10247000129788E594E00E9420378EE095E00E9454
:10248000203760E070E0CB010E946C3784E195E07A
:102490000E942037C701B6010E946C378AE195E09F
:1024A0000E942037C501B4010E946C3780E295E09C
:1024B0000E9420374AE06D857E858F8598890E942D
:1024C000213787E295E00E94203769817A818B81EC
:1024D0009C810E946C378DE295E00E9420376985CF
:1024E0007A858B859C850E946C3783E395E00E94FA
:1024F00020376D817E818F8198850E946C3789E3BA
:1025000095E00E94203781E095E00E94203789897C
:102510009A890E94623880ED93E00E94203796CF1E
:1025200062960FB6F894DEBF0FBECDBFDF91CF919C
:102530001F910F91FF90EF90DF90CF90BF90AF90E1
:102540009F908F907F906F905F904F903F902F90D3
:102550000895603E710508F0D8C3FB018827EC5749
:10256000FF4F8F4F0C94BA4E81E090E0A0E0B0E0B6
:102570008093320790933307A0933407B0933507C5
:10258000089510923607109237071092380710926C
:102590003907089510923A0710923B0710923C07B2
:1025A00010923D07089581E090E0A0E0B0E08093B4
:1025B0003E0790933F07A0934007B09341070895CB
:1025C0001092420710924307109244071092450759
:1025D000089583E090E0A0E0B0E0809346079093F8
:1025E0004707A0934807B0934907089588E790E00C
:1025F000A0E0B0E080935E0790935F07A093600730
:10260000B0936107089588E790E0A0E0B0E0809380
:10261000620790936307A0936407B09365070895DA
:1026200088E790E0A0E0B0E08093660790936707AA
:10263000A0936807B0936907089510926E071092EF
:102640006F07109270071092710708951092720729
:10265000109273071092740710927507089581E025
:1026600090E0A0E0B0E08093760790937707A09386
:102670007807B0937907089510927A0710927B0734
:1026800010927C0710927D07089510927E07109299
:102690007F07109280071092810708951092820799
:1026A0001092830710928407109285070895109264
:1026B000860710928707109288071092890708955D
:1026C00010928A0710928B0710928C0710928D0738
:1026D000089510928E0710928F0710929007109213
:1026E00091070895109296071092970710929807F5
:1026F00010929907089510929A0710929B071092D2
:102700009C0710929D07089510929E0710929F07B4
:102710001092A0071092A10708951092AE07109290
:10272000AF071092B0071092B10708951092B20748
:102730001092B3071092B4071092B5070895109243
:10274000B6071092B7071092B8071092B90708950C
:1027500081E090E0A0E0B0E08093C2079093C307CF
:10276000A093C407B093C507089581E090E0A0E06E
:10277000B0E08093C6079093C707A093C807B093B3
:10278000C90708958CE291E0A0E0B0E08093D607FD
:102790009093D707A093D807B093D90708958CE2F8
:1027A00091E0A0E0B0E08093DA079093DB07A0937C
:1027B000DC07B093DD0708958CE291E0A0E0B0E083
:1027C0008093DE079093DF07A093E007B093E107C3
:1027D00008951092E6071092E7071092E80710920A
:1027E000E90708951092EA071092EB071092EC07A0
:1027F0001092ED0708951092EE071092EF071092D5
:10280000F0071092F10708951092FE071092FF074B
:102810001092000810920108089510920208109278
:1028200003081092040810920508089581E090E0D2
:10283000A0E0B0E08093060890930708A0930808F2
:10284000B0930908089585E090E0A0E0B0E080939F
:102850000E0890930F08A0931008B09311080895E4
:1028600085E090E0A0E0B0E0809312089093130818
:10287000A0931408B0931508089589E190E0A0E0B2
:10288000B0E08093160890931708A0931808B093AF
:102890001908089582E390E0A0E0B0E08093260854
:1028A00090932708A0932808B0932908089582E3FD
:1028B00090E0A0E0B0E080932A0890932B08A093CA
:1028C0002C08B0932D08089582E390E0A0E0B0E0DA
:1028D00080932E0890932F08A0933008B09331086E
:1028E000089582E390E0A0E0B0E0809336089093F2
:1028F0003708A0933808B0933908089582E390E030
:10290000A0E0B0E080933A0890933B08A0933C0885
:10291000B0933D08089582E390E0A0E0B0E080939A
:102920003E0890933F08A0934008B0934108089553
:1029300080E991E0A0E0B0E080934E0890934F08CA
:10294000A0935008B0935108089580E991E0A0E069
:10295000B0E08093520890935308A0935408B0932A
:102960005508089580E991E0A0E0B0E08093560812
:1029700090935708A0935808B0935908089510925F
:102980005E0810925F081092600810926108089526
:102990001092620810926308109264081092650801
:1029A00008951092660810926708109268081092B5
:1029B00069080895109276091092770910927809A3
:1029C00010927909089510927A0910927B09109259
:1029D0007C0910927D09089510927E0910927F095A
:1029E000109280091092810908951092C6081092E1
:1029F000C7081092C8081092C90808951092CA0812
:102A00001092CB081092CC081092CD080895109225
:102A1000CE081092CF081092D0081092D1080895D5
:102A20001092D6081092D7081092D8081092D908A0
:102A300008951092DA081092DB081092DC081092C8
:102A4000DD0808951092DE081092DF081092E00869
:102A50001092E108089585E090E0A0E0B0E0809356
:102A6000EE089093EF08A093F008B093F108089552
:102A700085E090E0A0E0B0E08093F2089093F30846
:102A8000A093F408B093F508089585E090E0A0E0E5
:102A9000B0E08093F6089093F708A093F808B093FD
:102AA000F908089584EB95E1A0E0B0E08093FE087A
:102AB0009093FF08A0930009B0930109089584EB57
:102AC00095E1A0E0B0E08093020990930309A09300
:102AD0000409B0930509089584EB95E1A0E0B0E006
:102AE0008093060990930709A0930809B0930909F8
:102AF000089585E090E0A0E0B0E0809316099093FF
:102B00001709A0931809B0931909089585E090E07A
:102B1000A0E0B0E080931A0990931B09A0931C09D0
:102B2000B0931D09089585E090E0A0E0B0E08093A7
:102B30001E0990931F09A0932009B09321090895BD
:102B4000109226091092270910922809109229093B
:102B5000089510922A0910922B0910922C091092B4
:102B60002D09089510922E0910922F091092300904
:102B700010923109089510923E0910923F09109267
:102B80004009109241090895109242091092430998
:102B90001092440910924509089510924609109226
:102BA0004709109248091092490908951092560A4F
:102BB0001092570A1092580A1092590A08958CE3FD
:102BC00090E0A0E0B0E080935A0A90935B0AA09353
:102BD0005C0AB0935D0A089581E090E0A0E0B0E067
:102BE00080935E0A90935F0AA093600AB093610A93
:102BF00008951092660A1092670A1092680A10925D
:102C0000690A08958CE390E0A0E0B0E080936A0A3E
:102C100090936B0AA0936C0AB0936D0A089581E0BB
:102C200090E0A0E0B0E080936E0A90936F0AA093CA
:102C3000700AB093710A089510927E0A10927F0A6A
:102C40001092800A1092810A08958CE390E0A0E02F
:102C5000B0E08093820A9093830AA093840AB09391
:102C6000850A089581E090E0A0E0B0E08093860AB4
:102C70009093870AA093880AB093890A08951092C6
:102C80008E0A10928F0A1092900A1092910A08955B
:102C90008CE390E0A0E0B0E08093920A9093930AD6
:102CA000A093940AB093950A089581E090E0A0E083
:102CB000B0E08093960A9093970AA093980AB093F5
:102CC000990A08951092A60A1092A70A1092A80ACB
:102CD0001092A90A08958CE390E0A0E0B0E0809300
:102CE000AA0A9093AB0AA093AC0AB093AD0A0895D8
:102CF00081E090E0A0E0B0E08093AE0A9093AF0A4C
:102D0000A093B00AB093B10A0895660F771F660FBB
:102D1000771FFB01EE5CF84F108211821282138242
:102D200008958FEF9FEF08954F925F926F927F9279
:102D30008F929F92AF92BF92CF92DF92EF92FF92CB
:102D4000CF93DF935B01EB01CC0FDD1FCE010E941F
:102D5000414D482E512C612C712CCE0101960E94C0
:102D6000414DC82ED12CE12CF12C8DE8A81AB108C8
:102D700083E0A816B10488F5CE0144960E94414D27
:102D8000882E912CA12CB12CCE0145960E94414D4C
:102D9000482F50E060E070E08FEF88169104A104A6
:102DA000B104A9F44F3F51056105710581F48FEF1E
:102DB000481651046104710481F48FEFC816D104E0
:102DC000E104F10451F46FEF7FEFCB012BC04038E9
:102DD0005105610571056CF0F6CF80E8C816D10485
:102DE000E104F10484F740E050E0BA01812C912C19
:102DF0005401FE2CED2CDC2CCC24C40CD51CE61C80
:102E0000F71C540199248824C80CD91CEA1CFB1C0B
:102E1000742F662755274427CB01BA016C0D7D1D01
:102E20008E1D9F1DDF91CF91FF90EF90DF90CF908F
:102E3000BF90AF909F908F907F906F905F904F90DA
:102E400008950C9413470C9413470C9413470C9457
:102E500013470C9413474F925F926F927F928F9219
:102E60009F92AF92BF92CF92DF92EF92FF920F9319
:102E70001F93CF93DF9300D01F92CDB7DEB7FB0136
:102E80001689078982889388A684B784C284D384EC
:102E9000E484F58446805780608471844281538144
:102EA0006481758149835A836B837C830E9459288E
:102EB0001F921F921F920F931F93930182014981CA
:102EC0005A816B817C81BCD30F900F900F900F9033
:102ED0000F9080E090E00F900F900F900F90DF9197
:102EE000CF911F910F91FF90EF90DF90CF90BF9007
:102EF000AF909F908F907F906F905F904F900895CC
:102F000080918C0B81113FC081E080938C0B0E94DB
:102F10005928FC01E159FF4F2081222369F0709765
:102F200040815181628173814F5F5F4F6F4F7F4F4F
:102F30004083518362837383FC01E751FF4F2081FB
:102F4000222369F0709740815181628173814F5FC4
:102F50005F4F6F4F7F4F4083518362837383FC01C8
:102F6000ED59FE4F2081222361F07097808191817D
:102F7000A281B3810196A11DB11D80839183A2839B
:102F8000B38310928C0B08950F931F93CF93DF930D
:102F90008B01EA01AB01415051094433510508F05E
:102FA000D4C02230310508F0D0C048E3429FF00180
:102FB000439FF00D1124E60FF71FE80FF91F81E082
:102FC0008083232B11F46C2F07C061E0802F0E94B7
:102FD000580C209739F460E0802F0E94190C80E093
:102FE00090E0B5C0CF3FD10509F4ADC0F801E95379
:102FF000FB4FE4918E2F90E0FC013197E231F10517
:1030000008F09DC08827EC59FE4F8F4F0C94BA4EA4
:1030100084B5806884BDC7BDE2CF84B5806284BDBD
:10302000C8BDDDCF80918000806880938000D09300
:103030008900C0938800D3CF809180008062809304
:103040008000D0938B00C0938A00C9CF809180000C
:10305000886080938000D0938D00C0938C00BFCF98
:103060008091B00080688093B000C093B300B7CF68
:103070008091B00080628093B000C093B400AFCF65
:1030800080919000806880939000D0939900C093C5
:103090009800A5CF80919000806280939000D0939B
:1030A0009B00C0939A009BCF809190008860809392
:1030B0009000D0939D00C0939C0091CF8091A00080
:1030C00080688093A0008091A0008F7B8093A000F7
:1030D000D093A900C093A80082CF8091A000806205
:1030E0008093A000D093AB00C093AA0078CF8091CA
:1030F000A00088608093A000D093AD00C093AC0086
:103100006ECF80912001806880932001D0932901A7
:10311000C093280164CF80912001806280932001B8
:10312000D0932B01C0932A015ACF8091200188604F
:1031300080932001D0932D01C0932C0150CFC03833
:10314000D1050CF448CF61E047CF81E090E0DF91FA
:10315000CF911F910F91089580918F0B9091900BBB
:10316000892BA1F480E790E00E947E46FC01F9964D
:103170009C0123593F4FDF01D8971C921192E2170F
:10318000F307C9F79093900B80938F0B80918F0B6F
:103190009091900B0895683671050CF050C065361B
:1031A00071050CF08CC06C32710554F569327105F3
:1031B0000CF085C06831710594F46F3071050CF026
:1031C0007EC06630710544F4623071050CF077C042
:1031D000672B09F072C073C06B5071096BC062320B
:1031E00071053CF46F3171050CF069C069517109CA
:1031F00061C0645271096230710508F05EC05FC041
:103200006A3371057CF4673371050CF058C06D3278
:1032100071050CF452C0603371050CF450C0635357
:10322000710948C0643471053CF4613471050CF0D7
:1032300046C06D5371093EC0675471093BC0603987
:103240007105F4F46D387105D4F56637710564F4D1
:1032500063377105A4F5693671057CF16C3671052B
:1032600074F16F56710926C06038710534F46D37FA
:1032700071052CF5695771091DC0635871091AC091
:10328000603D710564F46D3C7105CCF461397105E4
:10329000A4F0643971059CF0695C71090BC06A3D4A
:1032A000710534F4673D710554F4635D710902C022
:1032B0006D5D71096330710510F080E0089581E063
:1032C0000895EF92FF920F931F93CF93DF9300D057
:1032D0001F92CDB7DEB78B017B01EE0CFF1C622F76
:1032E000C70129833A834B835C830E94494D29811E
:1032F0003A814B815C81992757FD9A95852F742FD0
:10330000632FC70101960E94494D0D58110929816B
:103310003A814B815C8103301105A8F4BA019927E9
:1033200077FD9095892FC70144960E94494D2981C8
:103330003A814B815C81652F772788279927C701C0
:1033400045960E94494D80E090E00F900F900F90BD
:103350000F90DF91CF911F910F91FF90EF90089503
:10336000CF92DF92EF92FF92CF93DF93EB0113DFC7
:10337000882359F1FE01EE0FFF1FEE0FFF1FEE5CD9
:10338000F84FC080D180E280F3808FE395E00E9407
:10339000203781E095E00E94203783E495E00E9489
:1033A0002037CE010E94623881E095E00E942037EC
:1033B00085E495E00E942037C701B6010E946C3772
:1033C0000E94FB070E94050704C089E894E00E9460
:1033D000203780E090E0DF91CF91FF90EF90DF9079
:1033E000CF900895EF92FF920F931F93CF93DF93A7
:1033F00080918D0B90918E0B892B09F066C084E033
:1034000090E00E947E46EC0160E070E08DDC1616D4
:1034100017067CF100E010E0B801CE01BCDE882385
:1034200019F0B801CE0195D80F5F1F4F013E11056D
:1034300099F792E3E92E97E0F92E00E010E0B80149
:10344000CE01A9DE882341F0F7012081318142813C
:103450005381B801CE0135DF0F5F1F4FF4E0EF0E4F
:10346000F11C0639110559F7D0938E0BC0938D0BC3
:103470002CC082E3E82E87E0F82E00E010E0B801CF
:10348000CE0189DE8823C1F0B801CE014DDCF70101
:1034900060837183828393836F3F7F4F8F4F9F4FF2
:1034A00059F4B801CE0155D8F7012081318142810C
:1034B0005381B801CE0105DF0F5F1F4FF4E0EF0E1F
:1034C000F11C013E1105D9F6CFCF80918D0B909163
:1034D0008E0BDF91CF911F910F91FF90EF90089588
:1034E0004F925F926F927F928F929F92AF92BF9214
:1034F000CF92DF92EF92FF920F931F93CF93DF93C0
:1035000000D01F92CDB7DEB76DDF40900E0850900F
:103510000F08609010087090110864DF8090120806
:1035200090901308A0901408B09015080E94FB0713
:10353000C090BA0AD090BB0AE090BC0AF090BD0AD5
:103540000E94FB07C701B6010E942B4C6B017C0156
:10355000C301B2010E942B4C9B01AC01C701B60113
:103560000E94194E2B013C016091BE0A7091BF0A66
:103570008091C00A9091C10A0E942B4C6B017C0182
:10358000C501B4010E942B4C9B01AC01C701B601DF
:103590000E94194EAB01BC0149835A836B837C8323
:1035A0000E9459281F921F921F921F921F92812CD6
:1035B000912CA12CB12CC12CD12C760149815A819E
:1035C0006B817C818A019B01B301A20139D00E94E9
:1035D00059281F921F921F921F921F9297018601D6
:1035E000B301A2012DD00E9459281F921F921F9251
:1035F0001F921F9297018601B701A60121D00FB635
:10360000F894DEBF0FBECDBF80E090E00F900F902A
:103610000F900F90DF91CF911F910F91FF90EF903E
:10362000DF90CF90BF90AF909F908F907F906F90E2
:103630005F904F900895089508950895089508950E
:103640002F923F924F925F926F927F928F929F92B2
:10365000AF92BF92CF92DF92EF92FF920F931F93A0
:10366000CF93DF93CDB7DEB7E4970FB6F894DEBF04
:103670000FBECDBF1C012A013B010F83188729878C
:103680003A872C960EAD1FAD2C97FC01E55AFD4FE5
:1036900060817181828193810E942B4C9B01AC01DE
:1036A000C301B2010E948A4C0E94814E6B8B7C8BBD
:1036B0008D8B9E8BF101E15AFD4F6081718182817A
:1036C00093810E942B4C9B01AC016F817885898589
:1036D0009A850E948A4C0E94814E6F8B788F898FC9
:1036E0009A8FF101ED59FD4F608171818281938143
:1036F0000E942B4C9B01AC01C701B6010E948A4C71
:103700000E94814E6B8F7C8F8D8F9E8F0E94D70C75
:103710006D877E878F87988BF101E452FE4F11826F
:1037200010823296118210823E96A114B10461F08B
:10373000C501A0E0B0E040815181628173818417AE
:103740009507A607B70714F0A080B180F101E051FA
:10375000FE4F8114910461F0C401A0E0B0E040810B
:1037600051816281738184179507A607B70714F00A
:1037700080809180F101EC50FE4F0115110561F040
:10378000C801A0E0B0E0408151816281738184175B
:103790009507A607B70714F0008111819101205FFA
:1037A0003F4F3A8B298BC501A0E0B0E0F10180A723
:1037B00091A7A2A7B3A72101FAE84F0E511CA12C93
:1037C000B12CD20158968D929D92AD92BC925B978E
:1037D0003101BCEF6B1ABEEF7B0A20E030E0F30151
:1037E000008F118F228F338F0E94FB070E94FB07EF
:1037F0000E94FB070E94FB074091BA0A5091BB0A46
:103800006091BC0A7091BD0A49AB5AAB6BAB7CAB03
:103810000E94FB078091BE0A9091BF0AA091C00A46
:10382000B091C10A8F839887A987BA870E94FB0746
:103830008090C20A9090C30AA090C40AB090C50AB2
:10384000F101E959FD4F10821182128213823496E0
:103850001082118212821382349610821182128297
:10386000138234961182108232961182108232961F
:1038700011821082329649A95AA96BA97CA940836A
:1038800051836283738334968F819885A985BA8525
:1038900080839183A283B383349680829182A282B3
:1038A000B3822D96EFAC2D970B891C892D893E890B
:1038B00089899A890E945F0E2E96EFAC2E970F8908
:1038C000188D298D3A8D4F81588569857A85C20179
:1038D0000E945F0E2F96EFAC2F970B8D1C8D2D8DB8
:1038E0003E8DB501A401C3010E945F0ED101519626
:1038F0001C92F101E557FF4F1082E658FF4F1082EE
:10390000C1010E94D639C1010E94DA3989899A8998
:103910000E942C39C2010E942C39C3010E942C390B
:10392000F101ED51FE4FFAA3E9A381E090E091830C
:1039300080837101FBE1EF1AFEEFFF0AD7018D933F
:103940009C93810109511E4FF8019183808341E0CE
:1039500050E069897A89C1010E940F27D7014D91F2
:103960005C91B201C1010E940F27F8014081518191
:10397000B301C1010E940F2711E0F101EE53FD4F89
:10398000108389899A890E944C0EC2010E944C0EB4
:10399000C3010E944C0E64E670E080E090E00E945B
:1039A0009F0CC10180529E4FDC011C9311961C9309
:1039B000A1014E515E4FFA0110832D96FFAD2D9758
:1039C000F1110FC02E962FAD2E97211105C02F9605
:1039D0003FAD2F97332339F1910121593F4FF90121
:1039E00010822E96FFAD2E97F11105C0910127513F
:1039F0003F4FF90110822F96FFAD2F97F11105C0AF
:103A000091012D593E4FF90110822D962FAD2D9722
:103A1000FC0120832E963FAD2E973C932F96EFAD61
:103A20002F97DA01EC9389899A890E940610C201C6
:103A30000E940610C3010E94061089899A890E947B
:103A40005C0FC2010E945C0FC3010E945C0F0E94C8
:103A5000FB07DC011C968C918B8B18861F82F10171
:103A6000E052FE4FF88FEF8B91012F513E4F3C8F6C
:103A70002B8FA1014E515E4F58A34F8FC1018D5125
:103A80009E4F98A78FA3D101AB51BE4FBAA7A9A74C
:103A90003796FCA7EBA7275531403CA32BA34E5DDF
:103AA00051095EA34DA3225C3F4F3EA72DA7425C68
:103AB0005F4F58AB4FA7EF89F88D808181110BC004
:103AC000AB8DBC8D8C91811106C0EF8DF8A18081EA
:103AD000882309F463C3FB89F11160C3C1010E940B
:103AE000B4394FA158A569897A89C1010E94682714
:103AF00049A55AA5B201C1010E9468274BA55CA542
:103B0000B301C1010E94682789899A890E94C60F62
:103B1000C2010E94C60FC3010E94C60FC1018E5888
:103B20009F4F9C878B87DC018C91882349F1898981
:103B30009A890E9406104101BDE58B1ABDEF9B0AD0
:103B40005101E9E6AE1AEDEFBE0A6101FEE4CF1ABB
:103B5000FDEFDF0A71012BE7E21A2DEFF20A810176
:103B600007581D4F910129593D4FA10142585E4F01
:103B700069897A89C1010E94E130AB85BC851C92BC
:103B8000F101E451FF4FFC87EB878081882339F1F5
:103B9000C2010E9406104101FCE58F1AFDEF9F0A49
:103BA000510125E6A21A2DEFB20A61013CE4C31AC5
:103BB0003DEFD30A710147E7E41A4DEFF40A8101A2
:103BC00003581D4F910125593D4FA10146565E4FA7
:103BD000B201C1010E94E130AB85BC851C92F101AC
:103BE000EA59FE4FFC87EB878081882339F1C301B6
:103BF0000E9406104101FBE58F1AFDEF9F0A51015B
:103C000021E6A21A2DEFB20A61013AE4C31A3DEF90
:103C1000D30A710143E7E41A4DEFF40A81010F570B
:103C20001D4F910121593D4FA1014A545E4FB301EF
:103C3000C1010E94E130AB85BC851C928101015914
:103C40001F4FF80180818823E9F1EE5DFD4F60810F
:103C50007181072E000C880B990B0E942B4C9B0145
:103C6000AC01F101E959FD4F60817181828193813D
:103C70000E94B24E181634F5D8011C9268E574E023
:103C800081010E521E4FC8010E94DA3861E875E0CA
:103C9000C8010E94DA3860ED73E0C8010E94DA388A
:103CA0002D96BFAD2D97BB2309F470C3C101825877
:103CB0009E4F0E946738F101E25BFF4F1082118234
:103CC00012821382810107511F4FD8018C918823E2
:103CD00009F43EC0F101ED56FD4F60817181072E60
:103CE000000C880B990B0E942B4C9B01AC01F1013D
:103CF000E559FD4F60817181828193810E94B24EAE
:103D0000181634F5D8011C9268E574E081010E5252
:103D10001E4FC8010E94DA3869EA75E0C8010E94A6
:103D2000DA3860ED73E0C8010E94DA382E96BFAD34
:103D30002E97BB2309F42FC3C10186569E4F0E94C4
:103D40006738EBA1FCA1FE961082118212821382C9
:103D500081010D591E4FF80180818823E9F1EE5C45
:103D6000FE4F60817181072E000C880B990B0E9419
:103D70002B4C9B01AC01F101E159FD4F6081718138
:103D8000828193810E94B24E181634F5D8011C929C
:103D900068E574E081010E521E4FC8010E94DA38B6
:103DA00061ED75E0C8010E94DA3860ED73E0C8018A
:103DB0000E94DA382F96BFAD2F97BB2309F4F0C2CB
:103DC000C1018A549E4F0E946738EDA1FEA1FE9664
:103DD000108211821282138260E089899A890E947E
:103DE000D50E882361F0F101E25BFF4F1082118252
:103DF00012821382C10182589E4F0E94673860E090
:103E0000C2010E94D50E882361F0ADA5BEA51D920A
:103E10001D921D921C921397C10186569E4F0E94BF
:103E2000673860E0C3010E94D50E882359F0EFA5E2
:103E3000F8A91082118212821382C1018A549E4F06
:103E40000E946738F101E159FF4F8081AF89B88D39
:103E50008C93E658FF4F8081EB8DFC8D8083F101C0
:103E6000ED59FE4F8081AF8DB8A18C93E551F140A3
:103E70004081518162817381EBA1FCA1FE9680801B
:103E80009180A280B380EDA1FEA1FE96C080D1807A
:103E9000E280F38049AB5AAB6BAB7CAB0E94FB0773
:103EA00049A95AA96BA97CA94093BA0A5093BB0AA5
:103EB0006093BC0A7093BD0A0E94FB078092BE0A01
:103EC0009092BF0AA092C00AB092C10A0E94FB075A
:103ED000C092C20AD092C30AE092C40AF092C50A04
:103EE000C1010E94D639EF89F88D8081882309F4B9
:103EF0004AC00E94D70C2D853E854F855889621790
:103F000073078407950760F40E94D70C2D853E85C2
:103F10004F8558896217730784079507A0F51EC05F
:103F20000E94D70C6B017C012D853E854F855889F9
:103F3000C21AD30AE40AF50AF101E15BFD4F2081C0
:103F4000318142815381A8EEB3E00E94734D6C151C
:103F50007D058E059F0508F428C2D6CF0E94D70C98
:103F60006B017C01F101E15BFD4F208131814281D8
:103F70005381A8EEB3E00E94734D6C157D058E054C
:103F80009F0508F412C2AB8DBC8D8C91882309F477
:103F90004AC00E94D70C2D853E854F8558896217EF
:103FA00073078407950760F40E94D70C2D853E8522
:103FB0004F8558896217730784079507A0F51EC0BF
:103FC0000E94D70C6B017C012D853E854F85588959
:103FD000C21AD30AE40AF50AF101ED5AFD4F208115
:103FE000318142815381A8EEB3E00E94734D6C157C
:103FF0007D058E059F0508F4EFC1D6CF0E94D70C32
:104000006B017C01F101ED5AFD4F2081318142812C
:104010005381A8EEB3E00E94734D6C157D058E05AB
:104020009F0508F4D9C1AF8DB8A18C91882309F4FC
:104030004AC00E94D70C2D853E854F85588962174E
:1040400073078407950760F40E94D70C2D853E8581
:104050004F8558896217730784079507A0F51EC01E
:104060000E94D70C6B017C012D853E854F855889B8
:10407000C21AD30AE40AF50AF101E95AFD4F208178
:10408000318142815381A8EEB3E00E94734D6C15DB
:104090007D058E059F0508F4B6C1D6CF0E94D70CCA
:1040A0006B017C01F101E95AFD4F20813181428190
:1040B0005381A8EEB3E00E94734D6C157D058E050B
:1040C0009F0508F4A0C185E99BE00E942A0A181602
:1040D00019068CF585E99BE00E94080A8F7D8534DE
:1040E000910549F567E475E0C1018E529E4F0E942B
:1040F000DA388EE493E00E9420370E94FB070E948A
:104100000507F101E159FF4F1082E658FF4F108279
:10411000E658FF4F1082AF89B88D1C92EB8DFC8D55
:104120001082AF8DB8A11C92B1E0BB8BE1E0F0E052
:10413000F887EF8304C02F813885232B81F06CE54D
:1041400075E0C1018E529E4F0E94DA38AF89B88D5A
:104150001C92EB8DFC8D1082AF8DB8A11C92C10119
:104160000E948436F101E252FE4F808191810196D6
:10417000918380838D3291400CF49DCCD101AA5261
:10418000BE4F8D919C911197892B09F094CC149678
:104190008D919C91892B09F44DC18DCC81010A52DE
:1041A0001E4FD8018D919C91892B21F0C1010E9455
:1041B0008436F7CF88E695E00E9420372D96BFAD74
:1041C0002D97BB2311F1EF81F885EF2BF1F4FB89DB
:1041D000F11142C08EE193E00E9420370E94FB075C
:1041E0000E9405072E962FAD2E97222381F18AE19A
:1041F00093E00E9420370E94FB070E9405072F963C
:104200003FAD2F9731111AC027C02E964FAD2E9774
:10421000442341F08F819885892B21F49B8991114A
:104220001BC0E5CF2F96AFAD2F97AA23A9F0EF8142
:10423000F885EF2B89F4FB89F1110EC086E193E03C
:104240000E9420370E94FB070E94050705C02F9699
:104250009FAD2F979111F2CF85E090E0A9A1BAA16F
:104260008D939C9391012B513E4F3E872D87D90111
:104270008D939C93810109511E4FF8019183808396
:1042800045E050E069897A89C101C9D5AD85BE850F
:104290004D915C91B201C101C2D5F80140815181BB
:1042A000B301C101BCD5C1010E94DE39F101E25B5D
:1042B000FF4F4081518162817381E658FF4FC0807A
:1042C000D180E280F380E658FF4F80809180A28009
:1042D000B38049AB5AAB6BAB7CAB0E94FB0749A9DF
:1042E0005AA96BA97CA94093BA0A5093BB0A609360
:1042F000BC0A7093BD0A0E94FB07C092BE0AD0920E
:10430000BF0AE092C00AF092C10A0E94FB078092A5
:10431000C20A9092C30AA092C40AB092C50AC1010F
:104320000E94D639C1010E94DA390E94FB070E941F
:104330005807C10105D6A9A1BAA11D921C92ED850D
:10434000FE8511821082D8011D921C9240E050E03F
:1043500069897A89C10163D5ED85FE8540815181E6
:10436000B201C1015CD5D8014D915C91B301C1018D
:1043700056D5C1010E94DE39BB89BB2309F457C160
:104380000E94FB0721E0FC01248751C1E1E0F0E03D
:10439000F887EF8397CCE1E0F0E0F887EF83D8CCA3
:1043A000E1E0F0E0F887EF8317CD6AE273E0810186
:1043B0000E521E4FC8010E94DA3860ED73E0C8014A
:1043C0000E94DA3869EF75E0C8010E94DA3822E00D
:1043D00030E038872F83D7CD66E273E081010E523B
:1043E0001E4FC8010E94DA3860ED73E0C8010E94D8
:1043F000DA386EE076E0C8010E94DA3842E050E038
:1044000058874F8310CE62E273E081010E521E4F37
:10441000C8010E94DA3860ED73E0C8010E94DA3802
:1044200063E276E0C8010E94DA3882E090E0988783
:104430008F8349CE11821082F101E452FE4F8081B8
:104440009181009749F46AE473E081010E521E4F96
:10445000C8010E94DA38C6C0019709F0D4C00E9492
:10446000FB078C01FC0180819181A281B381181628
:1044700019061A061B0644F081E090E0A0E0B0E0C7
:1044800080839183A283B383F80184819581A6817F
:10449000B781181619061A061B0644F081E090E051
:1044A000A0E0B0E084839583A683B783F80180857C
:1044B0009185A285B385181619061A061B0644F0C5
:1044C00081E090E0A0E0B0E080879187A287B38789
:1044D00062ED73E0CE0101960E9418396AEC74E037
:1044E000CE0101960E94DA386BED74E0CE010196A0
:1044F0000E94DA386091BA0A7091BB0A8091BC0AB6
:104500009091BD0A0E942B4C6B017C01D8016D91EA
:104510007D918D919C910E942B4C9B01AC01C70118
:10452000B6010E94194EAB01BC01CE0101960E945A
:10453000AA386BEE74E0CE0101960E94DA386091E1
:10454000BE0A7091BF0A8091C00A9091C10A0E9470
:104550002B4C6B017C01F801648175818681978108
:104560000E942B4C9B01AC01C701B6010E94194E61
:10457000AB01BC01CE0101960E94AA386BEF74E03A
:10458000CE0101960E94DA386091C20A7091C30A86
:104590008091C40A9091C50A0E942B4C6B017C014A
:1045A000D80118966D917D918D919C911B970E94D9
:1045B0002B4C9B01AC01C701B6010E94194EAB0107
:1045C000BC01CE0101960E94AA38BE016F5F7F4FE9
:1045D00081010E521E4FC8010E94E83889819A81DC
:1045E0000E9413470E94FB07BC01CE0101960E9466
:1045F000BF06BE016F5F7F4FC8010E94E838898106
:104600009A810E941347F101E452FE4F808191810B
:104610000196823091051CF49183808302C011823F
:104620001082F101E652FE4F1182108244CA86E7E1
:1046300095E00E9420378F8198850E94623880ED36
:1046400093E00E9420370E94FB072F81388530932A
:10465000310720933007C901E4960FB6F894DEBF06
:104660000FBECDBFDF91CF911F910F91FF90EF90C3
:10467000DF90CF90BF90AF909F908F907F906F9082
:104680005F904F903F902F900895CF92DF92EF92DE
:10469000FF920F931F93CF93DF937C016B018A01ED
:1046A000E9010E94F219F601EE0FFF1FEE0FFF1F46
:1046B000EE5CF84F80819181F701918380830E94A5
:1046C000F219000F111F000F111FF801EE5CF84FD7
:1046D00081E04081518162817381413051056105E2
:1046E000710509F080E0F70182870E94F219CC0F72
:1046F000DD1FCC0FDD1FCE5CD84F88819981AA8148
:10470000BB81F70182839383A483B58316821782CA
:1047100010861186DF91CF911F910F91FF90EF903E
:10472000DF90CF900895CF92DF92EF92FF920F9398
:104730001F93CF93DF93EC018AE190E09E8B8D8BEA
:104740008BE190E0988F8F8B89E190E09A8F898F31
:104750008FE090E09C8F8B8F8EE190E09E8F8D8F0D
:104760008EE090E098A38F8F85E490E09AA389A3D0
:1047700084E490E09CA38BA3FE01E657FF4F80E208
:1047800090E09683858381E290E0908787838FE134
:1047900090E0928781871486138616861586108A84
:1047A000178683E490E0928B818B82E490E0948B77
:1047B000838BE658FF4F83E290E09683858384E203
:1047C00090E09087878382E290E0928781871486C9
:1047D000138616861586108A178681E490E0928BE0
:1047E000818B80E490E0948B838BE152FF4F1182A8
:1047F0001082329611821082329611821082CE017E
:1048000083D5CE010E940C3ACE0182589E4F41E0E2
:1048100050E0FC01538F428FDE01A656BE4F24E0CC
:1048200030E05B963C932E935A976E01FAE4CF1AD0
:10483000FEEFDF0A28E030E0F601338F228F20E11F
:1048400030E0FC013183208321E130E03583248393
:104850002FEF3FEF33832283378326836285608780
:104860006385618767E170E011967C936E9368E1E0
:1048700070E015967C936E93149713963C932E9349
:10488000129717963C932E9316971A966C911A9737
:1048900018966C9318971B966C911B9719966C93AE
:1048A00019976DE170E0F601718360836CE170E04F
:1048B000758364833383228337832683628560878D
:1048C00063856187BE0168547D4FFB016081718102
:1048D0008E0104551D4FF801008111817E01FAE51A
:1048E000EF1AFDEFFF0AF701E080F180FC01F78A83
:1048F000E68A158B048B6130710519F4318F208F96
:1049000003C0FC01518F408FCE0186549D4FFC01A6
:10491000808191819E0122553D4FF9012081318195
:10492000AE0148555D4FFA014081518157965C9325
:104930004E93569755963C932E935497019719F49E
:104940008FEF9FEF02C081E090E059969C938E9389
:104950005897DE01A454BD4F8D919C9111971C97DF
:104960002D913C91C655DD4F48815981F601578BF9
:10497000468B358B248B019719F48FEF9FEF03C083
:1049800081E090E0F601918F808FDF91CF911F91B0
:104990000F91FF90EF90DF90CF9008952F923F926C
:1049A0004F925F926F927F928F929F92AF92BF923F
:1049B000CF92DF92EF92FF920F931F93CF93DF93EB
:1049C000CDB7DEB7CA57D1090FB6F894DEBF0FBE18
:1049D000CDBF8C01FC0110821182128213821482DD
:1049E0001582168217821086118612861386148607
:1049F0001586168617862C01F0E14F0E511CC20158
:104A00000E94503968018AE8C80ED11CC6010E9474
:104A100050397801ECEFEE1AEEEFFE0AC7010E9462
:104A200050393801F2E86F1AFEEF7F0AC3010E9485
:104A3000780D480186E6881A8EEF980AC4010E9414
:104A4000780D5801EAE4AE1AEEEFBE0AC5010E94E5
:104A5000780D62ED73E0C8018E529E4F0E941839A6
:104A6000F801E852FE4F11821082329611821082B4
:104A70003296118210823296118210823296108202
:104A800031961082319610823196118210823296C0
:104A900011821082329611821082329610823196E3
:104AA0001082319610823196108211821282138206
:104AB00034961082118212821382349610821182EF
:104AC00012821382349610821182128213823496DB
:104AD0001082118212821382349610821182128205
:104AE00013823496108211821282138234961082BD
:104AF00011821282138234961082118212821382E2
:104B0000349610821182128213823496108211829E
:104B1000128213823496108211821282138234968A
:104B200010821182128213823496108211821282B4
:104B3000138234961082118212821382349610826C
:104B40003196108231961082319610821182128233
:104B5000138234961082118212821382349610824C
:104B6000118212821382349610823196108231960D
:104B700010823196108231961082319610823196D1
:104B800010823196108231961082319610823196C1
:104B900010823196108231961082319610823196B1
:104BA00010823196108231961082319610823196A1
:104BB0001082319610823196108231961082319691
:104BC00010823196108231961082118212821382E5
:104BD00034961082118212821382349610821182CE
:104BE00012821382D801A55ABD4F8CE0EEE2F3E0A9
:104BF00001900D928A95E1F7F801E959FD4F108275
:104C000011821282138234961082118212821382D0
:104C1000349610821182128213823496118210828D
:104C20003296118210823296118210823296108250
:104C300011821282138234961082118212821382A0
:104C4000349610821182128213823496108211825D
:104C50001282138234961082118212821382349649
:104C6000108211821282138234961182108232963F
:104C70001182108232961182108232961082118235
:104C80001282138234961082118212821382349619
:104C90001082118212821382349610823196108211
:104CA00031961082319611821082329611821082D2
:104CB00032961182108232961182108232961182BF
:104CC00010823296118210823296118210823296B0
:104CD00011821082329611821082329611821082D5
:104CE000329611821082329611821082329611828F
:104CF00010823296118210821801FEE32F1AFDEF06
:104D00003F0AF1011082CE0101960E9450398AE7D4
:104D1000FE013196D20101900D928A95E1F7CE0104
:104D200001960E9450398AE7FE013196D601019022
:104D30000D928A95E1F7CE0101960E9450398AE7DB
:104D4000FE013196D70101900D928A95E1F788E531
:104D5000F801808B89E5F60180838AE5F70180837D
:104D6000CE0101960E94780D8CE1FE013196D301AF
:104D700001900D928A95E1F7CE0101960E94780D7F
:104D80008CE1FE013196D40101900D928A95E1F7F4
:104D9000CE0101960E94780D8CE1FE013196D5017D
:104DA00001900D928A95E1F7C801BDDCF1011082F6
:104DB000C658DF4F0FB6F894DEBF0FBECDBFDF91F0
:104DC000CF911F910F91FF90EF90DF90CF90BF9008
:104DD000AF909F908F907F906F905F904F903F909B
:104DE0002F9008950F931F93CF93DF938B01EA01C8
:104DF00086E493E00E94203781E095E00E9420370E
:104E0000F80180810E946137CE010E9462380E94C1
:104E1000FB07DF91CF911F910F910C940507CF9263
:104E2000DF92EF92FF920F931F93CF93DF93CDB753
:104E3000DEB728970FB6F894DEBF0FBECDBF8B014B
:104E40006A018E529E4F7C0162E473E00E94DA3860
:104E500061E075E0C7010E94DA38F801808189833A
:104E60001A8241E050E08E010F5F1F4FB801C70169
:104E70000E947D384AE0B801C6010E94D847F80177
:104E800001900020E9F73197AF01401B510BB801A9
:104E9000C7010E947D380E94FB07BC01C8010E9427
:104EA000BF06B801C7010E94E83889819A810E9433
:104EB000134728960FB6F894DEBF0FBECDBFDF9123
:104EC000CF911F910F91FF90EF90DF90CF900895B9
:104ED000FC01DB01AD59BF4F8C91882319F022E012
:104EE00030E002C020E030E0DB01AB59BF4F8C91D5
:104EF000882311F023E030E0DB01AC59BF4F8C91E7
:104F0000882311F024E030E0DB01AA59BF4F8C91D7
:104F1000882311F026E030E0DA018D919C91821710
:104F2000930721F091E0121613060CF090E0DA01DD
:104F30002D933C93992319F0A901CF0170CF0895C7
:104F40008F929F92AF92BF92CF92DF92EF92FF9299
:104F50000F931F93CF93DF93EC018EE393E00E94B6
:104F600020378BED94E00E9420376E0182E8C81A4A
:104F70008EEFD80AC6010E94580D0E942B4C4B019F
:104F80005C01FE01E55AFD4F608171818281938150
:104F90000E942B4C9B01AC01C501B4010E94194E2B
:104FA00042E00E9493378BEE94E00E9420377E010E
:104FB000E6E6EE1AEEEFFE0AC7010E94580D0E94C7
:104FC0002B4C4B015C01FE01E15AFD4F6081718168
:104FD000828193810E942B4C9B01AC01C501B401DD
:104FE0000E94194E42E00E9493378BEF94E00E949A
:104FF00020378E010A541E4FC8010E94580D0E948E
:105000002B4C4B015C01CD59DD4F688179818A8140
:105010009B810E942B4C9B01AC01C501B4010E94F5
:10502000194E42E00E9493370E94FB070E94050739
:105030008AE393E00E9420378BED94E00E942037B2
:10504000F601A08DB18D20893189428953890E9452
:105050007D4D0E946C378BEE94E00E942037F70163
:10506000A08DB18D20893189428953890E947D4D5F
:105070000E946C378BEF94E00E942037F801A08DDE
:10508000B18D20893189428953890E947D4D0E94CA
:105090006C370E94FB07DF91CF911F910F91FF901A
:1050A000EF90DF90CF90BF90AF909F908F900C9437
:1050B0000507CF93DF938091930B9091940B892BED
:1050C00051F483EC92E00E947E46EC0167DCD093C1
:1050D000940BC093930B8091930B9091940BDF9161
:1050E000CF910895CF93DF93EC012AEC30E04BECA5
:1050F00050E069EC70E0C9DA2EEC30E04FEC50E0A3
:105100006DEC70E0CE010C96C0DA24ED30E045ED98
:1051100050E063ED70E0CE014896B7DA28ED30E05C
:1051200049ED50E067ED70E0CE018496AEDA2EEDE9
:1051300030E04FED50E06DED70E0CE01C096DF91B4
:10514000CF91A3CACF93DF938091910B9091920B53
:10515000892BE9F48CE390E00E947E46EC01FC018F
:10516000CC96118210823C96E817F907D1F7198284
:1051700018821D861C86198E188E1DA21CA219AAC3
:1051800018AACE01AFDFD093920BC093910B809100
:10519000910B9091920BDF91CF910895EF92FF9236
:1051A0000F931F93CF93DF93162F072F7A0141158B
:1051B000510559F4862F0E94F10B31E020E0019750
:1051C00009F030E0C32FD22F26C04130510509F538
:1051D000262F663310F02AEC260F80917B00922F49
:1051E0009870877F892B80937B00277020642093A1
:1051F0007C0080917A00806480937A0080917A00AC
:1052000086FDFCCFC091780080917900D0E0D82B4A
:1052100002C0C0E0D0E082E0E816F10410F588E3B7
:1052200096E00E94203781E095E00E94203783E4D9
:1052300095E00E942037812F902F0E94623881E0F4
:1052400095E00E94203785E495E00E942037CE014A
:105250000E9462380E94FB070E94050780E090E0F0
:1052600002C081E090E0DF91CF911F910F91FF90FC
:10527000EF9008950F931F93CF93DF93FC0120814C
:10528000318121153105D9F1EC01822F0E94F10BFA
:1052900021E0892B09F420E02B876A85261729F065
:1052A0001E821F82188619860BC08E819F81A88559
:1052B000B9850196A11DB11D8E839F83A887B987EB
:1052C0000E811F81288539858A819B81AC81BD81B2
:1052D000081719072A073B0794F081E0682788819F
:1052E0000E94190C0990D881C02D0E94AC1840E092
:1052F00050E0BE01DF91CF911F910F914FCFDF9111
:10530000CF911F910F9108952F923F924F925F92EC
:105310006F927F928F929F92AF92BF92CF92DF92C5
:10532000EF92FF920F931F93CF93DF93CDB7DEB72A
:1053300060970FB6F894DEBF0FBECDBF988B8F87F6
:105340000E94F219EF85F889E751FE4F81E0409104
:10535000FE075091FF076091000870910108452BEE
:10536000462B472B09F480E080830E94F219EF85D9
:10537000F889E651FE4F81E0409102085091030800
:105380006091040870910508452B462B472B09F4C2
:1053900080E080830E94F219EF85F889E551FE4F85
:1053A00081E04091060850910708609108087091CB
:1053B0000908452B462B472B09F480E080830E9487
:1053C000F21980914E0890914F08A0915008B09129
:1053D0005108EF85F889E451FE4F80839183A283C1
:1053E000B3830E94F2198091520890915308A091C2
:1053F0005408B0915508EF85F889E051FE4F80833D
:105400009183A283B3830E94F219809156089091F0
:105410005708A0915808B0915908EF85F889EC50C9
:10542000FE4F80839183A283B3830E94F2198091FF
:10543000260890912708A0912808B0912908EF85A7
:10544000F889EC5FFD4F80839183A283B3830E9430
:10545000F21980912A0890912B08A0912C08B09104
:105460002D08EF85F889E85FFD4F80839183A28343
:10547000B3830E94F21980912E0890912F08A09179
:105480003008B0913108EF85F889E45FFD4F8083E3
:105490009183A283B3830E94F21980913608909180
:1054A0003708A0913808B0913908EF85F889E05F96
:1054B000FD4F80839183A283B3830E94F219809170
:1054C0003A0890913B08A0913C08B0913D08EF85C7
:1054D000F889EC5EFD4F80839183A283B3830E94A1
:1054E000F21980913E0890913F08A0914008B09138
:1054F0004108EF85F889E85EFD4F80839183A283A0
:10550000B3830E94F2198091D6079091D707A0919A
:10551000D807B091D907EF85F889E45EFD4F808305
:105520009183A283B3830E94F2198091DA0790914C
:10553000DB07A091DC07B091DD07EF85F889E05E1D
:10554000FD4F80839183A283B3830E94F2198091DF
:10555000DE079091DF07A091E007B091E107EF85AA
:10556000F889EC5DFD4F80839183A283B3830E9411
:10557000F219EF85F889E85DFD4F81E02091AE07D3
:105580003091AF072130310509F080E080830E941F
:10559000F219EF85F889E75DFD4F81E02091B207B0
:1055A0003091B3072130310509F080E080830E94FB
:1055B000F219EF85F889E65DFD4F81E02091B6078D
:1055C0003091B7072130310509F080E080830E94D7
:1055D000F219EF85F889EA5BFD4F81E0409186077B
:1055E000509187076091880770918907452B462B5A
:1055F000472B09F480E080830E94F219EF85F88937
:10560000E95BFD4F81E040918A0750918B076091E3
:105610008C0770918D07452B462B472B09F480E0B2
:1056200080830E94F219EF85F889E85BFD4F81E0E5
:1056300040918E0750918F0760919007709191076C
:10564000452B462B472B09F480E080830E94F219FA
:10565000EF85F889E75BFD4F81E040915E0850914E
:105660005F086091600870916108452B462B472BBD
:1056700009F480E080830E94F219EF85F889E65BE7
:10568000FD4F81E040916208509163086091640889
:1056900070916508452B462B472B09F480E08083E9
:1056A0000E94F219EF85F889E55BFD4F81E040919A
:1056B0006608509167086091680870916908452BE9
:1056C000462B472B09F480E080830E94F219EF8576
:1056D000F889E45BFD4F81E02091960730919707B0
:1056E0002130310509F080E080830E94F219EF85B6
:1056F000F889E35BFD4F81E020919A0730919B0789
:105700002130310509F080E080830E94F219EF8595
:10571000F889E25BFD4F81E020919E0730919F0761
:105720002130310509F080E080830E94F2198091D8
:105730005E0790915F07A0916007B0916107EF85C8
:10574000F889E15BFD4F80839183A283B3830E943C
:10575000F2198091620790916307A0916407B0915C
:105760006507EF85F889ED5AFD4F80839183A28309
:10577000B3830E94F2198091660790916707A09108
:105780006807B0916907EF85F889E95AFD4F808372
:105790009183A283B3830E94F219EF85F889E65CB6
:1057A000FD4F81E040916E0750916F076091700747
:1057B00070917107452B462B472B09F480E08083BD
:1057C0000E94F219EF85F889E55CFD4F81E0409178
:1057D0007207509173076091740770917507452B9C
:1057E000462B472B09F480E080830E94F219EF8555
:1057F000F889E45CFD4F81E040917607509177078E
:105800006091780770917907452B462B472B09F457
:1058100080E080830E94F219809166099091670967
:10582000A0916809B0916909EF85F889E55DFD4FA0
:1058300080839183A283B3830E94F21980916A09C5
:1058400090916B09A0916C09B0916D09EF85F88971
:10585000E15DFD4F80839183A283B3830E94F2199F
:1058600080916E0990916F09A0917009B0917109B2
:10587000EF85F889ED5CFD4F80839183A283B3832C
:105880000E94F219EF85F889E35CFD4F81E02091D9
:10589000C6073091C7072130310509F080E08083C9
:1058A000EF85F889E25CFD4F1082EF85F889E15CB5
:1058B000FD4F10820E94F219EF85F889E05CFD4FE0
:1058C00081E02091C2073091C3072130310509F0F2
:1058D00080E08083EF85F889EF5BFD4F1082EF85D4
:1058E000F889EE5BFD4F10820E94F219EF85F8896E
:1058F000ED5BFD4F81E02091E6073091E707213015
:10590000310509F080E080830E94F219EF85F88963
:10591000EC5BFD4F81E02091EA073091EB072130ED
:10592000310509F080E080830E94F219EF85F88943
:10593000EB5BFD4F81E02091EE073091EF072130C6
:10594000310509F080E080830E94F219EF85F88923
:10595000E95CFD4F81E02091760930917709213093
:10596000310509F080E080830E94F219EF85F88903
:10597000E85CFD4F81E020917A0930917B0921306C
:10598000310509F080E080830E94F219EF85F889E3
:10599000E75CFD4F81E020917E0930917F09213045
:1059A000310509F080E080830E94F2190F85188983
:1059B000055A1D4F80910E0890910F08A091100874
:1059C000B0911108F80180839183A283B3830E9470
:1059D000F219EF84F888F1EAEF1AFDEFFF0A8091DF
:1059E000120890911308A0911408B0911508F701BE
:1059F00080839183A283B3830E94F2198091160859
:105A000090911708A0911808B09119082F8538892E
:105A10002D593D4FF90180839183A283B383F8010F
:105A2000408151816281738114161506160617068E
:105A300044F041E050E060E070E0408351836283D5
:105A40007383F701408151816281738114161506B9
:105A50001606170644F041E050E060E070E0408335
:105A6000518362837383181619061A061B064CF0BD
:105A700081E090E0A0E0B0E0F90180839183A2830F
:105A8000B383D9018D909D90AD90BC90F701C080FB
:105A9000D180E280F380D8014D905D906D907C9034
:105AA0000E94FB07FC014082518262827382C482A1
:105AB000D582E682F78280869186A286B386EF85BC
:105AC000F889E95CFD4FB081B983EF85F889E55D20
:105AD000FD4F80819181A281B3814F8558894D5BB3
:105AE0005D4FFA01F081FB834F855889445B5D4F20
:105AF000FA01F081FA834F855889435C5D4FFA01C2
:105B0000F081FF834F855889405C5D4FFA01F08139
:105B1000F8874F855889475B5D4FFA01F081F98717
:105B20004F8558894A5B5D4FFA01F081FA87EF850E
:105B3000F889E85DFD4F2080EF85F889E751FE4F39
:105B40003080EF85F889E15BFD4F408151816281B2
:105B50007381EF85F889E45EFD4F00811181228118
:105B60003381EF85F889E05FFD4FC080D180E2800E
:105B7000F380EF85F889EC5FFD4F80809180A280F3
:105B8000B380EF85F889E451FE4F408051806280F8
:105B90007380EF85F88940A651A662A673A684A6F5
:105BA00095A6A6A6B7A6C0AAD1AAE2AAF3AA04AB54
:105BB00015AB26AB37AB40AF51AF62AF73AF34AE6E
:105BC00025AE2A8525A3398536A34A8147A340E41B
:105BD00050E060E070E0E05CFF4F408351836283FF
:105BE00073832885EF85F88926AF3F8137AFAF01F2
:105BF0004C5B5F4F2B81FA012083EF85F889EB5BCB
:105C0000FF4F80839183A283B383EF85F889E75B9D
:105C1000FF4F39813083AF85B88955968D919C911E
:105C200056978633910589F480E99BE0FD01E6589B
:105C3000FF4F918380833296118210828EE89BE021
:105C4000369691838083329630C08C33910589F4E7
:105C500088E89BE0EF85F889E658FF4F91838083C1
:105C6000EF85F889E458FF4F1182108286E89BE0A7
:105C700012C08E97E1F480E89BE0EF85F889E65842
:105C8000FF4F91838083EF85F889E458FF4F11829D
:105C900010828AE79BE0EF85F889EE57FF4F9183EA
:105CA0008083EF85F889EC57FF4F11821082EF85D2
:105CB000F889838D948D4A97D1F48CE89BE0E25863
:105CC000FF4F91838083EF85F889E058FF4F118261
:105CD00010828AE89BE0EF85F889EA57FF4F9183AD
:105CE0008083EF85F889E857FF4F11821082EF8596
:105CF000F889E85CFD4F20812983EF85F889E15D13
:105D0000FD4F4080518062807380EF85F889EC5BA5
:105D1000FD4F30813B83EF85F889E35BFD4F908138
:105D2000EF85F889E25CFD4F40814F83EF85F8896C
:105D3000EF5BFD4F50815887EF85F889E65BFD4F9B
:105D40008081EF85F889E95BFD4FA081AA87EF8507
:105D5000F889E75DFD4F2080EF85F889E651FE4F19
:105D60003080EF85F889ED5AFD4F208131814281E5
:105D700053812B873C874D875E87EF85F889E05EEE
:105D8000FD4F4081518162817381EF85F889EC5E1E
:105D9000FD4FC080D180E280F380EF85F889E85F15
:105DA000FD4F80809180A280B380EF85F889E6570F
:105DB000FF4F2F85388920513E4FD9010D911D91FC
:105DC0002D913C91008F118F228F338F848E958E71
:105DD000A68EB78EC0A2D1A2E2A2F3A244A355A37D
:105DE00066A377A32B853C854D855E8520A731A7CB
:105DF00042A753A734A625A63A85358B868B978B69
:105E000080E490E0A0E0B0E080AB91ABA2ABB3AB9C
:105E1000488546A75F8157A78B8184AB45AA56AAC0
:105E200067AA70AE998191AF85819681863391057D
:105E300089F480E99BE0AF85B889AC50BF4F8D9362
:105E40009C93AF85B889AA50BF4F1D921C928EE8D3
:105E50009BE026C08C33910589F488E89BE0AF85F0
:105E6000B889AC50BF4F8D939C93AF85B889AA5029
:105E7000BF4F1D921C9286E89BE012C08E97E1F402
:105E800080E89BE0AF85B889AC50BF4F8D939C9361
:105E9000AF85B889AA50BF4F1D921C928AE79BE03C
:105EA000AF85B889A450BF4F8D939C93AF85B889B7
:105EB000A250BF4F1D921C92838594854A97D9F4B6
:105EC0008CE89BE0EF85F889E850FF4F9183808351
:105ED000EF85F889E650FF4F118210828AE89BE037
:105EE000EF85F889F39591838083EF85F889EE5FDC
:105EF000FE4F11821082EF85F889E75CFD4FA0818B
:105F0000A9832F8538892D5C3D4FD9018D919D91B5
:105F10000D90BC91A02D8B839C83AD83BE83EF85B8
:105F2000F889EB5BFD4FB081BA83EF85F889E25BBE
:105F3000FD4F20812F83EF85F889E15CFD4F308193
:105F40003887EF85F889EE5BFD4F40814987EF8503
:105F5000F889E55BFD4F2080EF85F889E85BFD4F10
:105F60003080EF85F889E65DFD4F3081EF85F88957
:105F7000E551FE4F2081EF85F889E95AFD4F808178
:105F80009181A281B381EF85F889EC5DFD4F40815D
:105F9000518162817381EF85F889E85EFD4FC08091
:105FA000D180E280F380EF85F889E45FFD4F808047
:105FB0009180A280B3800F8518890C5F1E4FEF85FA
:105FC000F889EC50FE4F4080518062807380F80168
:105FD000408E518E628E738E848E958EA68EB78E75
:105FE000C0A2D1A2E2A2F3A244A355A366A377A3C1
:105FF00080A791A7A2A7B3A724A735A7358A268A89
:106000002F81278B80E490E0A0E0B0E080AB91ABE3
:10601000A2ABB3AB298526A7388537A74A8144AB05
:106020008B819C81AD81BE8185AB96ABA7ABB0AFB8
:10603000298121AF858196818633910589F480E994
:106040009BE0EF85F889E259FE4F91838083EF85CD
:10605000F889E059FE4F118210828EE89BE026C03D
:106060008C33910589F488E89BE0EF85F889E25943
:10607000FE4F91838083EF85F889E059FE4F1182AE
:10608000108286E89BE012C08E97E1F480E89BE0E6
:10609000EF85F889E259FE4F91838083EF85F88977
:1060A000E059FE4F118210828AE79BE0EF85F88964
:1060B000EA58FE4F91838083EF85F889E858FE4FB8
:1060C00011821082D8011B968D919C911C974A9742
:1060D000E1F48CE89BE0EF85F889EE58FE4F918360
:1060E0008083EF85F889EC58FE4F118210828AE890
:1060F0009BE0EF85F889E658FE4F91838083EF851A
:10610000F889E458FE4F11821082EF85F889E65C29
:10611000FD4F20818F8598894096222319F00E9497
:106120004C0E02C00E943A0EEF85F889E55CFD4FE7
:1061300020818F85988986579F4F222319F00E94CE
:106140004C0E02C00E943A0EEF85F889E45CFD4FC8
:1061500080818823D9F0C80160960FB6F894DEBF1D
:106160000FBECDBFDF91CF911F910F91FF90EF90A8
:10617000DF90CF90BF90AF909F908F907F906F9067
:106180005F904F903F902F900C944C0EC8016096FA
:106190000FB6F894DEBF0FBECDBFDF91CF911F9138
:1061A0000F91FF90EF90DF90CF90BF90AF909F90B6
:1061B0008F907F906F905F904F903F902F900C94B6
:1061C0003A0E2F923F924F925F926F927F928F92F0
:1061D0009F92AF92BF92CF92DF92EF92FF920F9376
:1061E0001F93CF93DF9300D000D0CDB7DEB73B0134
:1061F0001A0129011C830B83FA82E982DE82CD8297
:10620000F4018081882309F474C0F901C080D18031
:10621000E280F38020E030E0A901C701B6010E94CE
:10622000B24E181674F4F5012081318142815381F8
:10623000C701B6010E94B44DF2016083718382836D
:106240009383F301E05AFF4F8081F101008D118D9E
:10625000C088D188E288F388E981FA8180809180C2
:10626000A280B380D801A7019601882341F00E9443
:106270007D4D681579058A059B0544F023C00E9471
:106280007D4D86169706A806B906E4F4F2018080D3
:106290009180A280B38020E030E04AEF56E4C5014F
:1062A000B4010E94254C87FF0DC020E030E040E89B
:1062B0005FE3C501B4010E94B54DF20160837183B3
:1062C00082839383D801A70196010E947D4DE981C5
:1062D000FA816083718382839383F301FE968081C8
:1062E0009181A281B381EB81FC8180839183A28320
:1062F000B383ED81FE8180819181892B49F0C101B9
:106300000E94580DF301FE9660837183828393830C
:1063100026960FB6F894DEBF0FBECDBFDF91CF91AA
:106320001F910F91FF90EF90DF90CF90BF90AF90B3
:106330009F908F907F906F905F904F903F902F90A5
:1063400008952F923F924F925F926F927F928F9219
:106350009F92AF92BF92CF92DF92EF92FF920F93F4
:106360001F93CF93DF93CDB7DEB7A9970FB6F894FD
:10637000DEBF0FBECDBF99A788A77C836B830E9429
:10638000842988A599A50E940C3A88A599A50E9400
:10639000D63988A599A50E94DA392B813C81213014
:1063A0003105C9F12230310509F467C0232B09F00A
:1063B00097C068A479A430E1630E711C48A559A563
:1063C00042585E4F5A874987E8A5F9A5EA5BFD4F19
:1063D0005081598B88A599A589599D4F9C878B879A
:1063E000A8A5B9A5AF56BD4FBD8BAC8BE8A5F9A547
:1063F000ED55FD4FF98FE88F28A539A52D513E4F5A
:10640000388B2F874DE850E05F8B4E8B85E190E015
:1064100098878F8368C068A479A49AE8690E711C74
:10642000A8A5B9A5A656BE4FBA87A987E8A5F9A51C
:10643000E95BFD4FB081B98BE8A5F9A5E559FD4FA2
:10644000FC87EB8728A539A52D563D4F3D8B2C8B1E
:1064500048A559A54C555D4F598F488F88A599A5DA
:106460008B519E4F988B8F87AEE8B0E0BF8BAE8B81
:10647000E6E1F0E0F887EF8336C068A479A4FCEF8A
:106480006F1AFEEF7F0A28A539A52A543E4F3A8796
:106490002987E8A5F9A5E85BFD4F3081398B48A530
:1064A00059A541595D4F5C874B8788A599A58B56A7
:1064B0009D4F9D8B8C8BA8A5B9A5AB55BD4FB98FB2
:1064C000A88FE8A5F9A5E951FE4FF88BEF872FE8D3
:1064D00030E03F8B2E8B47E150E058874F8303C05D
:1064E0008CE396E00CC0C3010E94FA0D811105C037
:1064F000C3010E94EA0D882369F08DEC96E0A0D4D8
:106500000E94FB0781E090E0909331078093300771
:1065100090E0E1C388E594E093D48BE696E090D4D4
:10652000D3018C91CED483E097E08AD480ED93E0C0
:1065300087D481E090E0EF85F8899183808341E002
:1065400050E0B30188A599A50E940F27C3010E94BE
:106550004C0ED3019C968C918301005A1F4F8823C7
:1065600039F0C3010E94220E81E0D8018C9305C04E
:10657000C3010E940A0EF801108289859A850E9443
:10658000580DF301FE966083718382839383AB85FC
:10659000BC851D921D921D921C921397E8A5F9A52A
:1065A000E959FD4F1082118212821382E8A5F9A5E4
:1065B000E559FD4F1082118212821382E8A5F9A5D8
:1065C000E159FD4F108211821282138286E090E021
:1065D000EF85F8899183808346E050E0B30188A578
:1065E00099A50E940F2741E050E0B30188A599A525
:1065F0000E94F226212C312C210123948B819C8135
:106600008D559D4F28A539A5280F391F3B8B2A8B07
:106610004B815C81440F551F440F551F5E834D8392
:10662000CA0189569D4FA8A5B9A5A80FB91FBB8F50
:10663000AA8F8B819C81875A9E4F880F991FE8A54E
:10664000F9A5E80FF91FFF8FEE8FCA018B579D4FF9
:1066500028A539A5280F391F39A328A30C9748A5C9
:1066600059A5480F591F5BA34AA38D819E81895963
:106670009D4FA8A5B9A5A80FB91FBDA3ACA38D8137
:106680009E81E8A5F9A58E0F9F1F9C01205F3D4FBD
:106690003E872D8788A599A567D68A889B88AA8C6E
:1066A000BB8CCE8CDF8CE8A0F9A00AA11BA12CA189
:1066B0003DA149855A85B30188A599A582DD85E963
:1066C0009BE00E942A0A1816190624F01A821982E1
:1066D00010E01DC085E99BE00E94080A8F7D85348B
:1066E0009105A1F787E495E0ABD30E94FB0721E079
:1066F000DC011C962C938EE493E0A2D30E94FB074E
:106700000E940507E1E0F0E0FA83E98311E0C301AC
:106710000E94FA0D81111DC0C3010E94EA0D811172
:1067200018C0111116C0AC89BD896D917C91072EDE
:10673000000C880B990B0E942B4C9B01AC01EB8544
:10674000FC8560817181828193810E94254C87FD47
:106750006FC28BEA96E074D3C3010E94EA0D8111E7
:1067600064C242E050E0B30188A599A50E94F226D8
:1067700088E594E065D38BE696E062D3D3018C91F3
:10678000A0D382E796E05CD380ED93E059D3E98112
:10679000FA81EF2BD1F485E896E052D381E095E0C1
:1067A0004FD383E495E04CD38F8198858BD481E0DF
:1067B00095E046D385E495E043D3F9898F2F90E0A7
:1067C00081D40E94FB070E94050788A599A5EED5F4
:1067D00088A599A5EFD588E594E032D38BE696E0BD
:1067E0002FD3D3018C916DD389E896E029D380ED26
:1067F00093E026D3EB85FC851082118212821382EE
:10680000D3019C968C918301005A1F4F882331F04D
:10681000C3010E940A0EF801108206C0C3010E9443
:10682000220E81E0D8018C9389859A850E94580DAB
:10683000F301FE966083718382839383E8A5F9A5B3
:10684000E959FD4F1082118212821382E8A5F9A541
:10685000E559FD4F1082118212821382E8A5F9A535
:10686000E159FD4F108211821282138289859A8527
:106870000E94580D6A8F7B8F8C8F9D8F212C312C1D
:10688000210123948B819C818D559D4FE8A5F9A50D
:10689000E80FF91FFF8FEE8F8D819E8189569D4FE6
:1068A00028A539A5280F391F39A328A38B819C81DE
:1068B000875A9E4F880F991F48A559A5480F591F01
:1068C0005BA34AA38D819E818B579D4FA8A5B9A537
:1068D000A80FB91FBDA3ACA3ED81FE81E758FD4F02
:1068E000FFA3EEA38D819E8128A539A5820F931F5A
:1068F000AC01405F5D4F5B8B4A8BF1013197FE87A6
:10690000ED87F887EF8329813A81232B09F0C6C0F0
:1069100088A599A529D52D813E8129593D4F88A566
:1069200099A5280F391F8E8C9F8CA8A0B9A0CAA04A
:10693000DBA0ECA0FDA00EA11FA1080F191F498527
:106940005A85B3013EDC85E99BE00E942A0A1816AD
:10695000190614F010E01DC085E99BE00E94080AAA
:106960008F7D85349105B1F787E495E069D20E9467
:10697000FB0721E0DC011C962C938EE493E060D2AF
:106980000E94FB070E940507E1E0F0E0FA83E9833B
:1069900011E02D853E852A30310538F4AB85BC8564
:1069A0001D921D921D921C921397B989C301B111BA
:1069B0008DC10E94EA0D81116DC0112329F0ED8572
:1069C000FE85F887EF8366C0AC89BD896D917C91A7
:1069D000072E000C880B990B0E942B4C9B01AC01DD
:1069E000EB85FC8560817181828193810E94254CB9
:1069F00087FFE5CFC3010E94F30EAA89BB892D91C1
:106A00003D914D915C9160E573EC80E090E00E94D7
:106A1000574DC9010E94940CEA89FB89208131817C
:106A200042815381A3E0B0E00E94734D9B01AC0111
:106A3000C201B1010E94574D672B682B692B91F45D
:106A40008AE493E0FDD10E94FB070E94050788E5D8
:106A500094E0F6D18DE996E0F3D1C10133D380ED16
:106A600093E0EED1C3010E94D10DAA89BB892D917B
:106A70003D914D915C9160E573EC80E090E00E9467
:106A8000574DC9010E94940CBFEF2B1A3B0A4B0AC9
:106A90005B0A33CF8BEA96E0D3D104C041E050E0EB
:106AA0005A83498388E594E0CBD18BE696E0C8D140
:106AB000D3018C9106D28FEB96E0C2D180ED93E0AA
:106AC000BFD189859A850E94580DE88DF98DEF2BED
:106AD000A9F0DC01CB012A8D3B8D4C8D5D8D821B95
:106AE000930BA40BB50BB7FF07C0B095A09590957D
:106AF00081959F4FAF4FBF4F98878F8349815A81B0
:106B0000452B01F585E896E09BD181E095E098D191
:106B100083E495E095D18E899F89D4D281E095E078
:106B20008FD185E495E08CD1AF81B885BD01BB0FD5
:106B3000880B990B0E942B4C42E0F5D10E94FB0779
:106B40000E94050785E090E0EF85F88991838083B6
:106B500045E050E0B30188A599A50E940F27C30125
:106B60000E943A0E88A599A521D488A599A522D47A
:106B70002B813C8121303105B1F02230310521F1EA
:106B8000232B91F50E94FB074F815885CA01550FB1
:106B9000AA0BBB0B8093BA0A9093BB0AA093BC0AC2
:106BA000B093BD0A21C00E94FB07EF81F885CF0199
:106BB000FF0FAA0BBB0B8093BE0A9093BF0AA09352
:106BC000C00AB093C10A10C00E94FB072F8138850C
:106BD000C901330FAA0BBB0B8093C20A9093C30A5F
:106BE000A093C40AB093C50A0E94FB070E945807ED
:106BF000AF85B8891D921C9240E050E0B30188A592
:106C000099A50E940F2740E050E0B30188A599A5FF
:106C10000E94F2260E94FB07E981FA81F093310776
:106C2000E093300789819A8156C0B1E0B98B99CD44
:106C3000C3010E94F30EED85FE85208131814281E2
:106C4000538160E573EC80E090E00E94574DC901EC
:106C50000E94940CAD85BE852D913D914D915C9126
:106C6000A3E0B0E00E94734D9B01AC01C201B101F1
:106C70000E94574D672B682B692B39F48AE493E007
:106C8000DFD00E94FB070E940507C3010E94D10DBF
:106C9000AD85BE852D913D914D915C9160E573EC84
:106CA00080E090E00E94574DC9010E94940CBFEF14
:106CB0002B1A3B0A4B0A5B0AE981FA81EF2B09F494
:106CC000E9CC21E030E03A8329834BCD0E94FA0DD4
:106CD000811175CE72CEA9960FB6F894DEBF0FBEA5
:106CE000CDBFDF91CF911F910F91FF90EF90DF907B
:106CF000CF90BF90AF909F908F907F906F905F905C
:106D00004F903F902F900895CF93DF93FC01EA526C
:106D1000FE4F408151814115510551F1EC01C652A0
:106D2000DE4F288139818E529E4F24173507C8F4D3
:106D3000FC0180819181009761F0FC01E20FF31F5B
:106D400080818A3041F08D3029F480ED93E078D055
:106D500002C080E0B6D088819981019699838883AA
:106D600007C040E050E062ED73E038D2198218822B
:106D7000DF91CF910895CF92DF92EF92FF920F9320
:106D80001F93CF93DF936C017A018B01C0E0D0E0B9
:106D9000CE15DF0589F0D8016D918D01D601ED91F9
:106DA000FC910190F081E02DC6011995892B11F419
:106DB0007E0102C02196ECCFC701DF91CF911F91D8
:106DC0000F91FF90EF90DF90CF9008950E94A94F10
:106DD0000F931F93CF93DF93EC01888199810097E4
:106DE00029F02A813B812617370788F48B016F5FD2
:106DF0007F4F0E94C24E009761F0998388831B8366
:106E00000A832C813D81232B11F4FC01108281E047
:106E100001C080E0DF91CF911F910F9108950097FD
:106E200061F0FC0101900020E9F73197AF01481BA8
:106E3000590BBC0185E99BE09ECF80E090E008956E
:106E4000EECF8F929F92AF92BF920F931F93CF93EB
:106E5000DF93CDB7DEB7A1970FB6F894DEBF0FBEB4
:106E6000CDBF19A2423008F44AE08E010F5D1F4FDA
:106E7000842E912CA12CB12CA50194010E94834D4C
:106E8000E62FB901CA0101501109EA3014F4E05D9E
:106E900001C0E95CD801EC93232B242B252B61F74F
:106EA000C801BDDFA1960FB6F894DEBF0FBECDBFFF
:106EB000DF91CF911F910F91BF90AF909F908F90D6
:106EC0000895E091950BF091960B0190F081E02DE3
:106ED000682F85E99BE01994CF92DF92EF92FF92A1
:106EE000CF93DF9397FF17C06B017C018DE2E9DF41
:106EF000EC0166277727CB016C197D098E099F0964
:106F00004AE09FDF8C0F9D1FDF91CF91FF90EF90A4
:106F1000DF90CF9008954AE0DF91CF91FF90EF90FE
:106F2000DF90CF908ECF4F925F926F927F928F9231
:106F30009F92AF92BF92CF92DF92EF92FF926B013E
:106F40007C01B42E9B01AC010E94B64E882319F03F
:106F500082E297E027C026013701E89477F82FEF07
:106F60003FEF4FE75FE7C301B2010E94B64E8111C8
:106F70000DC02FEF3FEF4FE75FE7C301B2010E9463
:106F8000254C18161CF486E297E00CC02FEF3FEF5B
:106F90004FE75FE4C701B6010E94B24E18167CF4B9
:106FA0008AE297E0FF90EF90DF90CF90BF90AF9094
:106FB0009F908F907F906F905F904F9030CF2FEF8A
:106FC0003FEF4FE75FECC701B6010E94254C87FDFC
:106FD000E7CF20E030E0A901C701B6010E94254CAF
:106FE00087FF08C08DE26DDF4C01F7FAF094F7F8E7
:106FF000F09402C0812C912CA12C60E070E080E024
:107000009FE3AB1441F020E030E040E251E40E9405
:10701000194EA394F6CF9B01AC01C701B6010E94A3
:10702000B54D2B013C010E94864E6B017C010E94F4
:10703000294C9B01AC01C301B2010E94B44D2B014C
:107040003C014AE0C701B601FCDE7C01E80CF91CFA
:10705000BB2021F08EE235DFE80EF91EDB2CDD20AF
:1070600019F120E030E040E251E4C301B2010E9496
:107070008A4C2B013C010E94864E4B01A12CB12C65
:107080004AE0C501B401DDDEE80EF91EC501B40118
:107090000E94294C9B01AC01C301B2010E94B44D76
:1070A0002B013C01DA94DBCFC701FF90EF90DF901A
:1070B000CF90BF90AF909F908F907F906F905F9098
:1070C0004F900895BC01990F880B990B05CFCF9372
:1070D000DF93EC01188A198A1A8A1B8A60E086E11C
:1070E0000E94190C8A8D8295807F0E94920D61E02A
:1070F00086E1DF91CF910C94190CEF92FF920F93E0
:107100001F93CF93DF93FC012481358161157105B5
:1071100011F480E018C041155105A1F07B01EC018C
:107120008A01020F131FB80153DE882391F32881CF
:1071300039818C819D81B701820F931F0E94BF4FBF
:107140001D830C8381E0DF91CF911F910F91FF9000
:10715000EF900895EF92FF920F931F93CF93DF93D9
:10716000CDB7DEB764970FB6F894DEBF0FBECDBFC4
:107170007C01CB01BA018E010F5F1F4F22E044E07A
:107180000E945F46BC01FC0101900020E9F73197A5
:10719000AF01481B590BC701B0DF64960FB6F894D6
:1071A000DEBF0FBECDBFDF91CF911F910F91FF903A
:1071B000EF9008956115710549F0FB0101900020E1
:1071C000E9F73197AF01461B570B97CF80E0089541
:1071D000FB0144815581608171818FCFEF92FF92D5
:1071E0000F931F93CF93DF93EC017B018A01BA01C8
:1071F000EFDD2881398181110DC02115310519F08C
:10720000C9010E941347198218821D821C821B82A9
:107210001A8206C01D830C83B701C9010E94BF4FAB
:10722000CE01DF91CF911F910F91FF90EF900895C4
:10723000FC01118210821382128215821482611560
:10724000710549F0FB0101900020E9F73197AF018A
:10725000461B570BC3CF08950F931F93FC01EA5BA6
:10726000FF4F2081211110C03897008111812281A8
:1072700033813496408151816281738104171507EF
:10728000260737074CF404C0FC0124A5222321F073
:107290001F910F910C94220E1F910F910C940A0EC6
:1072A000FC011382128214821682158210861782C4
:1072B000128611861486138616861586108A1786FE
:1072C000128A118A148A138ADC01A15ABF4F1C92B8
:1072D00012AE13AE14AE15AE91971D921D921D9273
:1072E0001C92139714961D921D921D921C92139737
:1072F00014961C925A961C9211961C9212961C92ED
:1073000011961C9211961C9211961C9211961C9229
:1073100011961C9211961C92119684E59CE0119690
:107320009C938E93129611961C921E92129680E553
:107330009CE011969C938E93129611961C921E922D
:1073400012968CE49CE011969C938E931296119663
:107350001C921E92129688E49CE08D939C93E858B0
:10736000FF4F118210820895CF93DF93EC0183B118
:1073700083B1E0E0F1E080818081CE0182589E4FB0
:107380000E94990D83B183B180B180B1CE01865640
:107390009E4F0E94990D83B183B180B180B1CE011F
:1073A0008A549E4FDF91CF910C94990D0E94FB0758
:1073B0000C94D5080E94FB070C941707CF93DF931A
:1073C000EC01FC01EE53FD4F1082E858F109808179
:1073D000811104C0CE0140960E943A0EFE01E55C88
:1073E000FD4F8081811105C0CE0186579F4F0E94BD
:1073F0003A0EFE01E45CFD4F8081811105C0CE0193
:107400008C5F9E4F0E943A0E64E670E080E090E050
:10741000DF91CF910C949F0C2F923F924F925F92ED
:107420006F927F928F929F92AF92BF92CF92DF9294
:10743000EF92FF920F931F93CF93DF93EC010E9483
:10744000F219FE01EF56FD4F8091EE089091EF0882
:10745000918380830E94F219FE01ED56FD4F8091C9
:10746000F2089091F308918380830E94F219FE0143
:10747000EB56FD4F8091F6089091F7089183808339
:107480000E94F2198E0109561D4F609116097091E4
:10749000170980911809909119090E942B4CF80145
:1074A00060837183828393830E94F2191E01F5E643
:1074B0002F1AFDEF3F0A60911A0970911B09809104
:1074C0001C0990911D090E942B4CF101608371836E
:1074D000828393830E94F21920E030E048EC52E46A
:1074E000F80160817181828193810E94194E2B0184
:1074F0003C0120E030E048EC52E4F1016081718110
:10750000828193810E94194E4B015C0160911E099A
:1075100070911F0980912009909121090E942B4CA4
:1075200020E030E048EC52E40E94194E6B017C01EF
:107530002AE037ED43E25CE3C301B2010E94B24EA0
:1075400018168CF420E030E046EC52E4C301B2019E
:107550000E94254C87FD0FC0412C512C46EC642E17
:1075600042E4742E08C05AE0452E57ED552E53E2E2
:10757000652E5CE3752EF80140825182628273822F
:107580002AE037ED43E25CE3C501B4010E94B24E4C
:1075900018168CF420E030E046EC52E4C501B4014A
:1075A0000E94254C87FD0FC0812C912C26ECA22E29
:1075B00022E4B22E08C03AE0832E37ED932E33E258
:1075C000A32E3CE3B32EF10180829182A282B3828A
:1075D0002AE037ED43E25CE3C701B6010E94B24EF8
:1075E00018168CF420E030E046EC52E4C701B601F6
:1075F0000E94254C87FD0FC0C12CD12C86ECE82EB3
:1076000082E4F82E08C09AE0C92E97EDD92E93E2B5
:10761000E92E9CE3F92EFE01E156FD4FC082D18296
:10762000E282F3820E94F2198091D6089091D708E5
:10763000FE01EA55FD4F918380830E94F2198091EB
:10764000DA089091DB08FE01E855FD4F91838083B5
:107650000E94F2198091DE089091DF08FE01E65544
:10766000FD4F918380830E94F2198091FE089091D2
:10767000FF08FE01E455FD4F918380830E94F219BB
:107680008091020990910309FE01E255FD4F91831B
:1076900080830E94F2198091060990910709FE01EA
:1076A000E055FD4F918380830E94F2198091260955
:1076B00090912709FE01EE54FD4F918380830E9433
:1076C000F21980912A0990912B09FE01EC54FD4F8B
:1076D000918380830E94F21980912E0990912F0945
:1076E000FE01EA54FD4F918380830E94F21980913C
:1076F0003E0990913F09FE01E854FD4F918380833C
:107700000E94F2198091420990914309FE01E654CA
:10771000FD4F918380830E94F219809146099091D8
:107720004709FE01E454FD4F918380830E94F219C2
:107730008091C6089091C708A091C808B091C90867
:10774000FE01ED55FD4F0197A105B10519F481E04A
:10775000808301C010820E94F2198091CA08909122
:10776000CB08A091CC08B091CD08FE01EC55FD4F9F
:107770000197A105B10519F481E0808301C0108251
:107780000E94F2198091CE089091CF08A091D00864
:10779000B091D108CB55DD4F0197A105B10519F482
:1077A00081E0888301C01882DF91CF911F910F91F2
:1077B000FF90EF90DF90CF90BF90AF909F908F9011
:1077C0007F906F905F904F903F902F9008957894A6
:1077D00084B5826084BD84B5816084BD85B58260D6
:1077E00085BD85B5816085BD80916E008160809387
:1077F0006E001092810080918100826080938100F0
:1078000080918100816080938100809180008160FF
:10781000809380008091B10084608093B10080915A
:10782000B00081608093B00080919100826080936D
:1078300091008091910081608093910080919000EF
:107840008160809390008091A10082608093A1006C
:107850008091A10081608093A1008091A00081604F
:107860008093A0008091210182608093210180910A
:1078700021018160809321018091200181608093AA
:10788000200180917A00846080937A0080917A0050
:10789000826080937A0080917A00816080937A0080
:1078A00080917A00806880937A001092C10061E034
:1078B0008AE10E94580C61E08BE10E94580C61E063
:1078C00089E10E94580C61E08FE00E94580C61E051
:1078D0008EE10E94580C61E08EE00E94580C62E03C
:1078E00085E40E94580C62E084E40E94580C62E037
:1078F00080E10E94580C62E081E10E94580C61E036
:1079000080E20E94580C61E081E20E94580C61E024
:107910008FE10E94580C62E083E40E94580C62E000
:1079200082E40E94580C62E087E10E94580C62E0F9
:1079300088E10E94580C61E083E20E94580C61E0EB
:1079400084E20E94580C61E082E20E94580C62E0DE
:1079500081E40E94580C62E080E40E94580C62E0CE
:107960008DE10E94580C62E08CE10E94580C61E0AD
:1079700088E20E94580C61E089E20E94580C61E0A4
:1079800085E20E94580C61E085E20E94190C61E0DA
:107990008DE00E94580C61E089E00E94580C61E083
:1079A00088E00E94580C61E087E00E94580C61E07A
:1079B0008AE00E94580C61E08CE00E94580C62E062
:1079C0008FE30E94580C62E08BE30E94580C61E048
:1079D00084E00E94580C61E085E00E94580C61E050
:1079E00086E00E94580C61E087E00E94580C61E03C
:1079F00089E10E94190C61E08EE00E94190C61E09F
:107A00008FE10E94190C61E082E20E94190C62E091
:107A100081E30E94580C61E086E10E94580C61E00D
:107A200086E10E94190C8CB58F7D8CBD8CB5837F4F
:107A30008CBD8CB58C7F8CBD8DB58E7F8DBDCFB749
:107A4000F8948091C60A811127C0E6EBF4E0849196
:107A5000E0E7F4E09491E82FF0E0EE0FFF1FEF5D18
:107A6000FB4FA591B491EC91E92321F461E085E30A
:107A70000E94190C61E085E30E94580C8CB580616E
:107A80008CBD8CB580648CBD61E084E30E94580C91
:107A900061E083E30E94580C8091C60A8F5F809357
:107AA000C60ACFBFE091A50BF091A60B82E08083C0
:107AB000E091A10BF091A20B1082E091A30BF09149
:107AC000A40BD0E1D0831092AD0BE091A90BF09103
:107AD000AA0B86E08083E091A70BF091A80B808130
:107AE00080618083E091A70BF091A80B8081886072
:107AF0008083E091A70BF091A80B80818068808340
:107B0000E091A70BF091A80B80818F7D808364E6C4
:107B100070E080E090E00E949F0C0E9459280E9433
:107B200093230E94A2280E9472280E94D70C60937F
:107B30006B0B70936C0B80936D0B90936E0B80E8C6
:107B400097E190932F0780932E07C1E0C0936F00B9
:107B5000D093810010928000C093C90A80E092E027
:107B60009093C80A8093C70A9093870080938600F9
:107B700081E1809381001092810010928500109223
:107B800084008091C90A8061809381000E94D70C93
:107B90006093670B7093680B8093690B90936A0BEB
:107BA0000E94D70C60936F0B7093700B8093710BD6
:107BB0009093720B0E94D70C60936B0B70936C0BBD
:107BC00080936D0B90936E0B0E94F2198091820747
:107BD00090918307A0918407B09185070197A10533
:107BE000B105E1F48CE693E02BD90E945928CF939C
:107BF0001F921F921F921F92812C912CA12CB12CAD
:107C0000C12CD12C760197018601B701A6010E94F3
:107C1000201B0F900F900F900F900F900E94F21961
:107C200080917E0790917F07A0918007B091810796
:107C30000197A105B105E9F484E893E001D90E9418
:107C400059281F9221E02F931F921F921F92812C7F
:107C5000912CA12CB12CC12CD12C7601970186013D
:107C6000B701A6010E94201B0F900F900F900F905C
:107C70000F900E94F21980917A0790917B07A09152
:107C80007C07B0917D070197A105B105E9F48CE966
:107C900093E0D6D80E9459281F921F9221E02F937B
:107CA0001F921F92812C912CA12CB12CC12CD12C74
:107CB000760197018601B701A6010E94201B0F9053
:107CC0000F900F900F900F9084EB93E0B9D88FE74F
:107CD000282E82E0382E95E7A92E92E0B92E0E9438
:107CE000592842DB0E94D70C60936F0B7093700B86
:107CF0008093710B9093720B00916B0B10916C0B36
:107D000020916D0B30916E0B6017710782079307FE
:107D100048F460936B0B70936C0B80936D0B909396
:107D20006E0B2CC0DC01CB01801B910BA20BB30BA3
:107D3000883E9340A105B10508F108511C4F2F4F13
:107D40003F4F00936B0B10936C0B20936D0B309394
:107D50006E0B0E94A228EC010E943A29CE010C96DB
:107D60000E943A29CE0148960E943A29CE01849673
:107D70000E943A29CE01C0960E943A2985E99BE0EB
:107D80000E942A0A892B09F496C50E94D70C609399
:107D9000670B7093680B8093690B90936A0B85E96E
:107DA0009BE00E94080A8093660B982F9F7D953474
:107DB00079F02091640B3091650BF901EE5CF44F82
:107DC00080832F5F3F4F3093650B2093640B06C079
:107DD0000E94FB0721E0DC011C962C938091640B30
:107DE0009091650B8133910564F02AE02093660B36
:107DF000FC01EE5CF44F208301969093650B809319
:107E0000640B8091660B2091640B3091650B8A3076
:107E100039F4C9010197AFEFBAE0E2E3FBE004C037
:107E200022333105B4F747C5AF0142535B404817D1
:107E300059071CF441914D93F7CFFC01E150F54FE8
:107E40001082223031050CF432C589E093E00E94A3
:107E5000203781E095E00E94203783ED93E00E9477
:107E600020378FEF9AE00E94203783ED93E00E9445
:107E7000203780ED93E00E9420378AE390E03ED7E0
:107E8000EC011A821B821C821D821E821F821886B0
:107E900019861A861B861C861D861E861F86188AD2
:107EA000198A1A8A1B8A1C8A1D8A1E8A1F8A188EA2
:107EB000198E1A8E1B8E1C8E1D8E1E8E1F8E18A262
:107EC00019A21AA21BA21CA21DA21EA21FA218A6C2
:107ED00019A61AA61BA61CA61DA61EA61FA618AA92
:107EE00019AA1AAA1BAA1CAA1DAA1EAA1FAA18AE62
:107EF00019AE68E072E08FEF9AE00E94AE478C0105
:107F0000FC0180818654823008F027C165ED73E062
:107F1000C8010E94B64F892B09F4D3C068ED73E005
:107F2000C8010E94B64F892B09F4CBC06CED73E0F9
:107F3000C8010E94B64F892B09F4C6C06FED73E0EB
:107F4000C8010E94B64F892B09F4BEC063EE73E0EE
:107F5000C8010E94B64F892B09F4B9C067EE73E0DF
:107F6000C8010E94B64F892B09F4B4C06BEE73E0D0
:107F7000C8010E94B64F892B09F4ACC06EEE73E0C5
:107F8000C8010E94B64F892B09F4A7C062EF73E0C5
:107F9000C8010E94B64F892B09F4A2C066EF73E0B6
:107FA000C8010E94B64F892B09F49DC06AEF73E0A7
:107FB000C8010E94B64F892B09F498C06EEF73E098
:107FC000C8010E94B64F892B09F493C062E074E0A7
:107FD000C8010E94B64F892B09F48EC066E074E098
:107FE000C8010E94B64F892B09F489C06AE074E089
:107FF000C8010E94B64F892B09F484C06EE074E07A
:10800000C8010E94B64F892B09F47FC062E174E079
:10801000C8010E94B64F892B09F47AC066E174E06A
:10802000C8010E94B64F892B09F475C06AE174E05B
:10803000C8010E94B64F892B09F470C06EE174E04C
:10804000C8010E94B64F892B09F46BC062E274E04C
:10805000C8010E94B64F892B09F466C066E274E03D
:10806000C8010E94B64F892B09F461C06AE274E02E
:10807000C8010E94B64F892B09F45CC06EE274E01F
:10808000C8010E94B64F892B09F457C062E374E01F
:10809000C8010E94B64F892B09F452C066E374E010
:1080A000C8010E94B64F892B09F44DC06AE374E001
:1080B000C8010E94B64F892B09F448C08FEF9FEF8B
:1080C00047C080E090E044C081E090E041C08CE196
:1080D00090E03EC08DE690E03BC08FE690E038C077
:1080E00080E790E035C081E790E032C082E790E021
:1080F0002FC083E790E02CC084E790E029C088E798
:1081000090E026C089E790E023C08AE790E020C095
:1081100083E890E01DC084E890E01AC08DE890E00C
:1081200017C08EE890E014C08FE890E011C080E99D
:1081300090E00EC081EA90E00BC085EB90E008C0B3
:1081400086EB90E005C087EB90E002C088EB90E002
:108150009093010280930002BBC08FEF9FEF90933A
:10816000010280930002B8C0D8018C91883539F49F
:10817000C8010196F0D66A837B838C839D83F801C6
:108180008081893539F4C8010196E5D66E837F83F5
:1081900088879987D8018C918A3539F4C80101966E
:1081A000DAD66A877B878C879D87F8018081813446
:1081B00049F4C8010196CFD60E94814E6E877F8711
:1081C000888B998BD8018C91823449F4C80101962F
:1081D000C2D60E94814E6A8B7B8B8C8B9D8BF80163
:1081E0008081833449F4C8010196B5D60E94814E3E
:1081F0006E8B7F8B888F998FD8018C91833539F462
:10820000C8010196A8D66A8F7B8F8C8F9D8FF8014D
:108210008081803549F4C80101969DD60E94814E27
:108220006E8F7F8F88A399A3D8018C91863549F4EE
:10823000C801019690D60E94814E6AA37BA38CA3AD
:108240009DA3F8018081873549F4C801019683D642
:108250000E94814E6EA37FA388A799A7D8018C9115
:10826000853449F4C801019676D60E94814E6AA7EA
:108270007BA78CA79DA7F8018081843549F4C801AC
:10828000019669D60E94814E6EA77FA788AB99ABF5
:10829000D8018C918D3449F4C80101965CD60E94B6
:1082A000814E6AAB7BAB8CAB9DABF8018081813595
:1082B00049F4C80101964FD60E94814E6EAB7FAB48
:1082C00088AF99AF6EE374E080E090E047D68C0110
:1082D0000115110509F048CF0E94FB07DC011C962F
:1082E0008C900E94F219409046075090470760908A
:1082F000480770904907CEA8DFA8E8ACF9AC0E9407
:10830000FB07C092B60AD092B70AE092B80AF09280
:10831000B90A00910002109101029924939402304D
:10832000110530F0C8018F569109069708F0912C7D
:10833000882081F00D36110509F432C4C801885730
:1083400091098330910548F1CD97039730F18DEF76
:1083500092E0A5C2209719F489EF92E0A0C20F3FE6
:10836000BFEF1B07C9F301151105C9F48091CA0AB3
:108370009091CB0A892B61F482E090E0BFD421E197
:1083800032E0FC01318320839093CB0A8093CA0AA8
:10839000E090CA0AF090CB0A52C02097E9F20C3163
:1083A0001105B9F48091CC0A9091CD0A892B61F422
:1083B00082E090E0A3D42BE132E0DC012D933C93EA
:1083C0009093CD0A8093CC0AE090CC0AF090CD0A2D
:1083D0006AC00D361105B9F48091CE0A9091CF0A8A
:1083E000892B61F482E090E089D425E232E0FC013F
:1083F000318320839093CF0A8093CE0AE090CE0AF7
:10840000F090CF0A50C00F361105B9F48091D00A10
:108410009091D10A892B61F482E090E06FD42FE231
:1084200032E0DC012D933C939093D10A8093D00AE3
:10843000E090D00AF090D10A50C0E12CF12C003726
:108440001105B9F48091D20A9091D30A892B61F475
:1084500082E090E053D429E332E0FC0131832083B1
:108460009093D30A8093D20AE090D20AF090D30A74
:1084700068C001371105B9F48091D40A9091D50AEA
:10848000892B61F482E090E039D423E432E0DC010E
:108490002D933C939093D50A8093D40AE090D40A0C
:1084A000F090D50A68C002371105B9F48091D60A58
:1084B0009091D70A892B61F482E090E01FD42DE4DB
:1084C00032E0FC01318320839093D70A8093D60A4F
:1084D000E090D60AF090D70A66C003371105B9F4C8
:1084E0008091D80A9091D90A892B61F482E090E0BA
:1084F00005D427E532E0DC012D933C939093D90A13
:108500008093D80AE090D80AF090D90A64C0043762
:108510001105B9F48091DA0A9091DB0A892B61F494
:1085200082E090E0EBD321E632E0FC01318320834E
:108530009093DB0A8093DA0AE090DA0AF090DB0A83
:1085400064C008371105B9F48091DC0A9091DD0A06
:10855000892B61F482E090E0D1D32BE632E0DC019C
:108560002D933C939093DD0A8093DC0AE090DC0A23
:10857000F090DD0A64C009371105A9F48091DE0A84
:108580009091DF0A892B51F482E090E0B7D3FC018F
:10859000B182A0829093DF0A8093DE0AE090DE0A27
:1085A000F090DF0A66C00A371105A9F48091E00A4D
:1085B0009091E10A892B51F482E090E09FD3DC0195
:1085C0002D923C929093E10A8093E00AE090E00AB9
:1085D000F090E10A68C00D381105B9F48091E20A03
:1085E0009091E30A892B61F482E090E087D329E837
:1085F00032E0FC01318320839093E30A8093E20A06
:10860000E090E20AF090E30A68C00E381105B9F470
:108610008091E40A9091E50A892B61F482E090E070
:108620006DD3E3E9F2E0DC01ED93FC939093E50A6E
:108630008093E40AE090E40AF090E50A68C00F38FD
:108640001105B9F48091E60A9091E70A892B61F44B
:1086500082E090E053D3EDE9F2E0DC01ED93FC938E
:108660009093E70A8093E60AE090E60AF090E70A22
:1086700068C000391105B9F48091E80A9091E90ABF
:10868000892B61F482E090E039D3E7EAF2E0DC0183
:10869000ED93FC939093E90A8093E80AE090E80A4E
:1086A000F090E90A68C0013A1105B9F48091EA0A2C
:1086B0009091EB0A892B61F482E090E01FD3E1EB0B
:1086C000F2E0DC01ED93FC939093EB0A8093EA0ACD
:1086D000E090EA0AF090EB0A67C0053B1105B9F497
:1086E0008091EC0A9091ED0A892B61F482E090E090
:1086F00005D3EBEBF2E0DC01ED93FC939093ED0AF4
:108700008093EC0AE090EC0AF090ED0A4DC0063B35
:108710001105B9F48091EE0A9091EF0A892B61F46A
:1087200082E090E0EBD2E5ECF2E0DC01ED93FC932B
:108730009093EF0A8093EE0AE090EE0AF090EF0A31
:1087400033C0073B1105B9F48091F00A9091F10A0A
:10875000892B61F482E090E0D1D2EFECF2E0DC0111
:10876000ED93FC939093F10A8093F00AE090F00A65
:10877000F090F10A19C0083B1105B1F48091F20A9A
:108780009091F30A892B61F482E090E0B7D2E3EE96
:10879000F2E0DC01ED93FC939093F30A8093F20AEC
:1087A000E090F20AF090F30AE114F10489F489EF01
:1087B00092E00E9420370E94FB070E94050782E496
:1087C00094E00E940F3780ED93E00E940F376DC058
:1087D00085EF92E00E9420370E94FB070E94050768
:1087E0000E94FB07109231071092300700E010E062
:1087F0000F5F1F4F0130110541F081EF92E00E94A1
:1088000020370E94FB070E940507D701ED91FC91DC
:108810000480F581E02DBE01C70119950E94FB0778
:10882000C0903007D09031070E94FB07FC0184857F
:1088300001151105E9F281110AC0041515053CF472
:10884000C114D10421F0F2E0CF16D10489F685E9F4
:108850009BE00E942A0A181619062CF485E99BE071
:108860000E94080AF4CFCD2809F484C1992009F4A4
:1088700084C10E94F2198091420790914307A09110
:108880004407B09145070197A105B10509F075C1ED
:108890000E94FB0721E0DC011C962C936EC10E9414
:1088A00020370E94FB070E940507CE01BCD2109220
:1088B000650B1092640B8091FE0A811170C00E94BA
:1088C000FB07FC018485882309F469C00E945928AC
:1088D000EC01FC01EE53FD4F108240960E943A0ECF
:1088E000CE0186579F4F0E943A0ECE018C5F9E4F5D
:1088F0000E943A0E0E94AC187C018C01075C1F4F4D
:10890000C1E0D0E06801F8E3CF1AD108D6018C911C
:108910008823D9F088E594E00E9420378CE594E024
:108920000E942037CE010E94623880ED93E00E94C1
:10893000203760E08C2F0E94190C40E050E0BE010F
:10894000C7010E94CE28F6011082D8018C9188239D
:10895000F9F088E594E00E94203783E794E00E94D4
:108960002037CE010E94623880ED93E00E942037CC
:1089700061E08C2F0E94580C60E08C2F0E94190C33
:1089800041E050E0BE01C7010E94CE28F8011082EC
:1089900021960F5F1F4FC533D10509F0B3CF0E9459
:1089A000FB07DC011C968C918093FE0AC091FC0AA7
:1089B000D091FD0A0E94F219FC0182819381C817AF
:1089C000D90799F00E94F219DC0112968D919C91C1
:1089D00013979093FD0A8093FC0A0E9459280E94E5
:1089E00093230E94A2280E9472280E94D70C6093B1
:1089F000F80A7093F90A8093FA0A9093FB0A00919F
:108A0000670B1091680B2091690B30916A0B60170E
:108A100071078207930708F4A0C0DC01CB01801B1B
:108A2000910BA20BB30B89389341A105B10508F452
:108A30009EC00E94FB07DC011C968C91882319F0D4
:108A400085E093E002C081E093E00E9420370E941D
:108A5000FB070E9405070E945928EC01FC01ED5517
:108A6000FD4F8081882341F0CE0182589E4F0E94A5
:108A7000580D6B017C0107C0FE01E25BFF4FC08017
:108A8000D180E280F3800E94FB07C092BA0AD092A4
:108A9000BB0AE092BC0AF092BD0AFE01EC55FD4F04
:108AA0008081882341F0CE0186569E4F0E94580D4A
:108AB0006B017C0107C0FE01E853FF4FC080D180ED
:108AC000E280F3800E94FB07C092BE0AD092BF0AE8
:108AD000E092C00AF092C10AFE01EB55FD4F808181
:108AE000882341F0CE018A549E4F0E94580D6B019D
:108AF0007C0106C0CE5BDE4FC880D980EA80FB8057
:108B00000E94FB07C092C20AD092C30AE092C40A34
:108B1000F092C50A0E94FB070E9458070E9459283C
:108B20000E94A0270E94FB070E94D5080E94FB0715
:108B30000E9417078091F40A9091F50AA091F60A15
:108B4000B091F70A0196A11DB11D8093F40A90938C
:108B5000F50AA093F60AB093F70A0E94D70C609327
:108B6000670B7093680B8093690B90936A0B0E945C
:108B7000C70AB5C88DEE92E002C089EE92E00E946D
:108B800020370E94FB070E9405070E94FB071092F6
:108B9000B60A1092B70A1092B80A1092B90A85CE96
:108BA000209709F019CCD8CB8091C90C9091CA0CB0
:108BB0003AC11092980B1092970B88EE93E0A0E0C8
:108BC000B0E08093990B90939A0BA0939B0BB0937A
:108BD0009C0B86E593E09093960B8093950B85EC28
:108BE00090E09093A20B8093A10B84EC90E0909383
:108BF000A40B8093A30B80EC90E09093A60B809342
:108C0000A50B81EC90E09093A80B8093A70B82ECCE
:108C100090E09093AA0B8093A90B86EC90E0909340
:108C2000AC0B8093AB0B1092AE0B1092AF0B10926B
:108C3000B00B1092B10B8091C20C803320F09FEFEB
:108C40009093C30C11C08093C30C282F30E0F9011E
:108C5000EE0FFF1F2E0F3F1FF901EE5CF34F28EBC5
:108C60003BE0328321838F5F803390F48093C60C86
:108C7000282F30E0F901EE0FFF1F2E0F3F1FF901E3
:108C8000EE5CF34F28EB3BE0328321838F5F03C020
:108C90009FEF9093C60C8093C20C82E090E02ED0A0
:108CA00028E633E0FC01318320839093D00C80933D
:108CB000CF0C62ED73E089EC9CE00C941839EF92D4
:108CC0000F931F93CF93DF93E80147FD02C034E079
:108CD00001C034E1E42F440FFF0BF7FF03C0F1950F
:108CE000E195F109E32E022F2E2FAE01B3D1CE0173
:108CF000DF91CF911F910F91EF900895CF93DF9364
:108D00008230910510F482E090E0E091D50CF09172
:108D1000D60C20E030E0C0E0D0E0309711F1408187
:108D2000518148175907C0F04817590761F48281EB
:108D30009381209719F09B838A832BC09093D60C44
:108D40008093D50C26C02115310519F04217530721
:108D500018F49A01BE01DF01EF010280F381E02DDA
:108D6000DCCF2115310509F1281B390B24303105E1
:108D700090F412968D919C9113976115710521F0D5
:108D8000FB019383828304C09093D60C8093D50C0F
:108D9000FD01329644C0FD01E20FF31F81939193D0
:108DA000225031092D933C933AC02091D30C30913D
:108DB000D40C232B41F4209104023091050230930E
:108DC000D40C2093D30C2091020230910302211580
:108DD000310541F42DB73EB740910602509107028C
:108DE000241B350BE091D30CF091D40CE217F30760
:108DF000A0F42E1B3F0B2817390778F0AC014E5F0B
:108E00005F4F2417350748F04E0F5F1F5093D40C67
:108E10004093D30C8193919302C0E0E0F0E0CF0146
:108E2000DF91CF9108950F931F93CF93DF93009716
:108E300009F48CC0FC013297138212820091D50C88
:108E40001091D60C0115110581F420813181820F1A
:108E5000931F2091D30C3091D40C2817390779F542
:108E6000F093D40CE093D30C71C0D80140E050E0F3
:108E7000AE17BF0750F412962D913C911397AD0198
:108E80002115310509F1D901F3CF9D01DA013383B1
:108E9000228360817181860F971F8217930769F47F
:108EA000EC0128813981260F371F2E5F3F4F318318
:108EB00020838A819B8193838283452B29F4F093BD
:108EC000D60CE093D50C42C01396FC93EE93129708
:108ED000ED01499159919E01240F351FE217F307C7
:108EE00071F480819181840F951F029611969C9355
:108EF0008E938281938113969C938E931297E0E0D8
:108F0000F0E0D80112968D919C911397009719F07B
:108F1000F8018C01F6CF8D919C9198012E5F3F4F07
:108F2000820F931F2091D30C3091D40C281739074E
:108F300069F4309729F41092D60C1092D50C02C027
:108F4000138212821093D40C0093D30CDF91CF9133
:108F50001F910F9108956627772709C241ED5CE0C4
:108F600000C0FA01A191B081009719F41097E1F0C7
:108F7000CD01DC01CD010D90002011F4C00113C022
:108F8000FB012191222319F02015D9F7F3CFFB0122
:108F90002191201519F41E92119606C02223C1F7C3
:108FA0000D900020A1F7D001FA01A193B08308959C
:108FB000BB274A3031F4992322F4BDE29095819584
:108FC0009F4F30C0BB272A3051F4992342F4BDE2B1
:108FD00090958095709561957F4F8F4F9F4F01C001
:108FE000BB27FA01A62F6217710581059105330B86
:108FF00030FB66F0AA27660F771F881F991FAA1FEC
:10900000A21710F0A21B63953850A9F7A05DAA33F0
:1090100008F0A95DA19336F7B111B1931082CA018E
:1090200004C4BB27FB015527AA27880F991FAA1F35
:10903000A41710F0A41B83955051B9F7A05DAA3373
:1090400008F0A95DA193009779F7B111B19311923E
:10905000CB01EBC34F925F926F927F929F92AF9240
:10906000BF92CF92DF92EF92FF920F931F93CF9315
:10907000DF93CDB7DEB729970FB6F894DEBF0FBEEA
:10908000CDBF6A01122FB02E2BE3201720F0FF2452
:10909000F394F00E02C0BCE3FB2E0F2D27E0AE01CF
:1090A0004F5F5F4FCAD2AC018981982F9970913080
:1090B00031F0E1FC06C0E0FE06C090E205C09DE292
:1090C00003C09BE201C090E0EE2DE07183FF3CC045
:1090D000911102C083E001C084E0811718F4212FB0
:1090E000281B01C020E0E1110BC0F601822F30E205
:1090F000882319F031938150FBCFC20ED11C20E0A0
:10910000992329F0D6019C93F60131966F01C6018F
:109110000396E2FE0AC03EE4D6013C9341E4119678
:109120004C93119712963C9306C03EE6F6013083AD
:1091300041E641833283FC01322F40E2332309F4BC
:1091400042C041933150FACF82FF44C0911102C016
:1091500083E001C084E0811718F4212F281B01C08F
:1091600020E0E1110BC0F601822F30E2882319F0D4
:1091700031938150FBCFC20ED11C20E0992329F0FE
:10918000D6019C93F60131966F01C6010396E2FE6B
:109190000BC039E4D6013C933EE411963C93119701
:1091A00036E412963C9307C039E6F60130833EE67A
:1091B000318336E63283FC01322F40E2332319F04B
:1091C00041933150FBCFFC01E20FF11D10828EEF75
:1091D0009FEFB7C0F1E0911101C0F0E06F2F70E098
:1091E0001416150624F49A012F5F3F4F02C021E0A8
:1091F00030E0260F371FBB2029F06B2D70E06F5F2A
:109200007F4F02C060E070E0260F371F612F70E0D3
:10921000261737071CF4121B212F01C020E03E2D1A
:10922000387159F4D601322F60E2332319F06D936F
:109230003150FBCFC20ED11C20E0FF2331F0D6010C
:109240009C93B6016F5F7F4F6B01E1110BC0F6017C
:10925000922F30E3992319F031939150FBCFC20E36
:10926000D11C20E09F2D940F3A81782F7071A72E8A
:1092700084FF03C0313309F49150191624F4993056
:1092800018F098E001C091E0E42F852F57FF02C04D
:10929000E0E080E06E2F782FE0E0F0E0AEE29A2E82
:1092A0003A01691A71082A01461A570A0B2D10E073
:1092B0001195019511096F3F8FEF780729F4D601B9
:1092C0009C92C60101966C014617570784F06616FA
:1092D00077066CF47F01E40CF51CA1E0B0E0AC0F64
:1092E000BD1FEA0EFB1ED7011196BC9002C090E391
:1092F000B92E615071093196C60101967C01601743
:10930000710724F0D601BC926C01D5CF64177507A4
:1093100041F4363320F4353321F4A11002C081E347
:10932000B82EF601B082F701822F90E2882319F05F
:1093300091938150FBCFF701E20FF11D108280E085
:1093400090E029960FB6F894DEBF0FBECDBFDF9137
:10935000CF911F910F91FF90EF90DF90CF90BF9032
:10936000AF909F907F906F905F904F9008956F9215
:109370007F928F929F92AF92BF92CF92DF92EF92A5
:10938000FF920F931F93CF93DF93EC017B01611545
:10939000710519F0DB018D939C938E010F5F1F4FB8
:1093A0007880872D90E021D2892B11F0E801F5CF4C
:1093B000BDE27B1205C00F5F1F4F7980C1E008C07E
:1093C000EBE27E1204C08E010E5F1F4F7980C0E079
:1093D0006801F1E0CF1AD10843E050E064EF72E099
:1093E000C6010BD2892BE9F4680122E0C20ED11C20
:1093F00045E050E06FEE72E0C601FFD1892B21F409
:10940000680187E0C80ED11CE114F10419F0D701FE
:10941000CD92DC92C111F9C060E070E080E89FE776
:10942000FDC043E050E06CEE72E0C601E6D1892B4E
:1094300051F4E114F10409F4EDC00E5F1F4FF70180
:1094400011830083E7C0680160E070E0CB0100E0B9
:1094500010E0F601D0EDD70DDA3050F52C2F226058
:10946000622E2C2F2870C2FF05C0211127C00F5F6C
:109470001F4F24C0222311F001501109A5E0B0E0D4
:109480009B01AC0130D34B015C01880C991CAA1CD8
:10949000BB1CC501B4016D0F711D811D911D683983
:1094A000A9E97A078A07A9E19A0740F0C66005C0D2
:1094B000DE3F51F4C3FD44C0C8606C2EBFEFCB1A31
:1094C000DB0A7080C62DC5CF2D2F2F7D2531C1F52C
:1094D00040814D3211F4C06106C04B3221F031960B
:1094E00021E030E006C03296D60111964C9122E080
:1094F00030E0A0EDA40FAA3018F0E21BF30B20C05F
:1095000040E050E04038BCE05B075CF49A01220F79
:10951000331F220F331F420F531F440F551F4A0F93
:10952000511D3196DF0111972C91A0EDA20FAA30A9
:1095300048F3C4FF03C0519541955109040F151F0D
:10954000C1FF07C0E114F10421F03197D701ED9379
:10955000FC937FD1C370C33019F06B017C0106C04E
:109560006B017C01F7FAF094F7F8F09420E030E01A
:10957000A901C701B60169D1882309F443C017FFC7
:1095800006C0119501951109CBE0D3E002C0C3E2FA
:10959000D3E05E01B8E1AB1AB1084601BE2DAF2D94
:1095A00090E2E92EF12C0E151F057CF0FE012591AD
:1095B000359145915491B4018B2F9A2FABD14B012A
:1095C000B82FA92F0E191F09EECF2497F594E79411
:1095D000CA15DB0541F76401EB2EFA2E8E2D880F9C
:1095E0008F2D881F8F3F41F020E030E0A901C70197
:1095F000B6012BD1811106C082E290E09093D80C85
:109600008093D70CC701B60109C060E070E080E824
:109610009FEF04C060E070E080EC9FE7DF91CF91A6
:109620001F910F91FF90EF90DF90CF90BF90AF9080
:109630009F908F907F906F900895283008F027E0DA
:109640003327DA01990F311D87FD9160009661057E
:10965000710539F432602E5F3D9330E32A95E1F7CE
:1096600008959F3F30F080387105610509F03C5F37
:109670003C5F3D93913008F08068911DDF93CF935C
:109680001F930F93FF92EF92192F987F9695E92FD2
:1096900096959695E90FFF27EF57FC4F99273327AB
:1096A000EE24FF24A701E70105900894079428F40D
:1096B000360FE71EF81E491F511D660F771F881FC2
:1096C000991F0694A1F70590079428F4E70EF81E59
:1096D000491F561FC11D770F881F991F661F0694CB
:1096E000A1F70590079428F4F80E491F561FC71FCD
:1096F000D11D880F991F661F771F0694A1F705904B
:10970000079420F4490F561FC71FD81F990F661FD3
:10971000771F881F0694A9F784911095177041F060
:10972000D695C79557954795F794E7941A95C1F73D
:10973000E7E2F3E068941590159135916591959164
:1097400005907FE27395E118F10A430B560BC90BA4
:10975000D009C0F7E10CF11E431F561FC91FD01DD1
:109760007EF4703311F48A95E6CFE894015030F01E
:10977000080F0AF40027021708F4202F2395022F60
:109780007A3328F079E37D932A95E9F710C07D9329
:109790002A9589F6069497956795379517951794A6
:1097A000E118F10A430B560BC90BD00998F0239529
:1097B0007E9173957A3308F070E37C932013B8F7A9
:1097C0007E9170617D9330F0839571E37D9370E3BA
:1097D0002A95E1F71124EF90FF900F911F91CF91FF
:1097E000DF91992787FD909508959111F6C08032F9
:1097F00019F089508550D0F70895FB01DC014150E4
:10980000504088F08D9181341CF08B350CF4805ED3
:10981000659161341CF06B350CF4605E861B611140
:1098200071F3990B0895881BFCCFDC01FC01672FB5
:1098300071917723E1F7329704C07C916D93708327
:109840006291AE17BF07C8F3089540D008F481E0D5
:109850000895E89409C097FB3EF490958095709523
:1098600061957F4F8F4F9F4F9923A9F0F92F96E96C
:10987000BB279395F695879577956795B795F111E1
:10988000F8CFFAF4BB0F11F460FF1BC06F5F7F4F7E
:109890008F4F9F4F16C0882311F096E911C0772390
:1098A00021F09EE8872F762F05C0662371F096E899
:1098B000862F70E060E02AF09A95660F771F881F68
:1098C000DAF7880F9695879597F90895990F00080C
:1098D000550FAA0BE0E8FEEF16161706E807F90782
:1098E000C0F012161306E407F50798F0621B730B1D
:1098F000840B950B39F40A2661F0232B242B252B9E
:1099000021F408950A2609F4A140A6958FEF811D40
:10991000811D08950BD07BC06CD028F071D018F059
:10992000952309F05DC062C01124A5C081D0A0F3C9
:10993000959FD1F3950F50E0551F629FF001729FE4
:10994000BB27F00DB11D639FAA27F00DB11DAA1F03
:10995000649F6627B00DA11D661F829F2227B00D50
:10996000A11D621F739FB00DA11D621F839FA00DDB
:10997000611D221F749F3327A00D611D231F849F2B
:10998000600D211D822F762F6A2F11249F57504082
:109990008AF0E1F088234AF0EE0FFF1FBB1F661F1D
:1099A000771F881F91505040A9F79E3F510570F0D6
:1099B00017C061C05F3FECF3983EDCF38695779566
:1099C0006795B795F795E7959F5FC1F7FE2B880FD1
:1099D000911D9695879597F9089599278827089559
:1099E00097F99F6780E870E060E008959FEF80EC52
:1099F000089500240A9416161706180609060895F5
:109A000000240A9412161306140605060895092E5A
:109A10000394000C11F4882352F0BB0F40F4BF2BC9
:109A200011F460FF04C06F5F7F4F8F4F9F4F089509
:109A300057FD9058440F551F59F05F3F71F04795FF
:109A4000880F97FB991F61F09F3F79F087950895E4
:109A5000121613061406551FF2CF4695F1DF08C003
:109A6000161617061806991FF1CF86957105610520
:109A700008940895E894BB2766277727CB0197F9C8
:109A80000895F999FECF92BD81BDF89A992780B5C6
:109A90000895262FF999FECF1FBA92BD81BD20BD32
:109AA0000FB6F894FA9AF99A0FBE01960895052E0A
:109AB00097FB16F400940FD057FD05D024D007FC77
:109AC00002D046F408C050954095309521953F4FFF
:109AD0004F4F5F4F089590958095709561957F4F9A
:109AE0008F4F9F4F089531D0A59F900DB49F900D3B
:109AF000A49F800D911D11240895B7FFF4CFF3DFCB
:109B0000821B930B0895A1E21A2EAA1BBB1BFD0119
:109B10000DC0AA1FBB1FEE1FFF1FA217B307E4074C
:109B2000F50720F0A21BB30BE40BF50B661F771FA4
:109B3000881F991F1A9469F7609570958095909584
:109B40009B01AC01BD01CF010895A29FB001B39F5D
:109B5000C001A39F700D811D1124911DB29F700D36
:109B6000811D1124911D08955058BB27AA270ED09E
:109B70004ECF3FDF30F044DF20F031F49F3F11F44F
:109B80001EF434CF0EF4E095E7FB2ACFE92F50DF27
:109B900080F3BA17620773078407950718F071F40A
:109BA0009EF568CF0EF4E0950B2EBA2FA02D0B0179
:109BB000B90190010C01CA01A0011124FF27591B12
:109BC00099F0593F50F4503E68F11A16F040A22F18
:109BD000232F342F4427585FF3CF46953795279589
:109BE000A795F0405395C9F77EF41F16BA0B620B88
:109BF000730B840BBAF09150A1F0FF0FBB1F661FCF
:109C0000771F881FC2F70EC0BA0F621F731F841F11
:109C100048F4879577956795B795F7959E3F08F037
:109C2000B3CF9395880F08F09927EE0F97958795F6
:109C300008950CD0ECCEE4DE40F0DBDE30F021F411
:109C40005F3F19F0CDCE511116CFD0CEF1DE98F393
:109C50009923C9F35523B1F3951B550BBB27AA27AD
:109C600062177307840738F09F5F5F4F220F331F1F
:109C7000441FAA1FA9F333D00E2E3AF0E0E830D0EB
:109C800091505040E695001CCAF729D0FE2F27D0EE
:109C9000660F771F881FBB1F261737074807AB07BC
:109CA000B0E809F0BB0B802DBF01FF2793585F4F31
:109CB0002AF09E3F510568F093CEDDCE5F3FECF376
:109CC000983EDCF3869577956795B795F7959F5FF6
:109CD000C9F7880F911D9695879597F90895E1E04A
:109CE000660F771F881FBB1F621773078407BA07A9
:109CF00020F0621B730B840BBA0BEE1F88F7E09504
:109D0000089504D06894B111B6CE089599DE88F014
:109D10009F5790F0B92F9927B751A0F0D1F0660F57
:109D2000771F881F991F1AF0BA95C9F712C0B13072
:109D300081F0A0DEB1E008959DCE672F782F8827AF
:109D4000B85F39F0B93FCCF3869577956795B395B1
:109D5000D9F73EF490958095709561957F4F8F4F20
:109D60009F4F0895B3DD08F48FEF0895AFDD880BA2
:109D7000990B0895EE0FFF1F881F8BBF0790F69178
:109D8000E02D19946F927F928F929F92AF92BF9223
:109D9000CF92DF92EF92FF920F931F93CF93DF93B7
:109DA000EC01009789F4CB01DF91CF911F910F91C6
:109DB000FF90EF90DF90CF90BF90AF909F908F90EB
:109DC0007F906F900C947E46FC01E60FF71F9C017C
:109DD00022503109E217F30708F4AAC0D9010D9106
:109DE0001C91119706171707A8F00530110508F404
:109DF0009DC0C80104978617970708F497C00250C2
:109E00001109061B170B019311936D937C93CF01DE
:109E10000AD88CC05B01A01AB10A4C01800E911EB9
:109E2000A091D50CB091D60C40E050E0E12CF12C83
:109E3000109709F44AC0A815B905D1F56D907C902A
:109E40001197630182E0C80ED11CCA14DB0480F1B3
:109E5000A3014A195B096A0182E0C80ED11C12965F
:109E6000BC9012971396AC91B5E0CB16D10440F09C
:109E7000B282A38351834083D9016D937C930AC03E
:109E80000E5F1F4FC301800F911FF90191838083E3
:109E9000EB2DFA2FE114F10431F0D7011396FC9366
:109EA000EE93129743C0F093D60CE093D50C3EC0CE
:109EB0008D919C9111974817590708F4AC017D01C9
:109EC00012960D90BC91A02DB3CF8091D30C9091A0
:109ED000D40C88159905E1F446175707C8F480910A
:109EE000020290910302009741F48DB79EB7409112
:109EF000060250910702841B950BE817F907C0F47E
:109F0000F093D40CE093D30CF901718360830EC0FD
:109F1000CB010E947E467C01009751F0A801BE0152
:109F20001CD0CE010E941347C70104C0CE0102C05D
:109F300080E090E0DF91CF911F910F91FF90EF9023
:109F4000DF90CF90BF90AF909F908F907F906F9059
:109F5000089581E090E0F89419C0FB01DC0102C093
:109F600001900D9241505040D8F70895FB01DC015B
:109F70008D91019080190110D9F3990B0895FB017F
:109F8000DC0101900D920020E1F7089512E0C2EA91
:109F9000D2E000E005C0802FFE01ECDE2196011D1D
:0E9FA000C33AD10780E00807B1F7F894FFCF6D
:109FAE00FFFF0000D90C8000200A0D000000000009
:109FBE00001E1B27172B17000000001D1B251770F6
:109FCE001A00000000BE068303CF0800000000BD8B
:109FDE00068103B70500000000BC067F038605005E
:109FEE00000000BB067D03550500000000BA067B8D
:109FFE00031C0500000000B9067903E3040000000D
:10A00E0000B8067703AA0400000000B7067503AB7C
:10A01E000800000000B6067303390400000000B506
:10A02E00067103480400000000B4066F03C7030066
:10A03E00000000B3066103850300000000B2066D48
:10A04E0003220400000000B1066B03E403000000CD
:10A05E0000B00669039B0300000000AF06670316FD
:10A06E000900000000AE066503A60800000000AD62
:10A07E000663039908000000001C1B2317911600AD
:10A08E000000001F1B29173808523033005230329F
:10A09E0000523037005230310052303900523837CA
:10A0AE0000523030005238370052303800362E30E1
:10A0BE002E312E46000052313300523132005231D1
:10A0CE00310052373300523732005237310001001F
:10A0DE000000010000000100000052383500523827
:10A0EE00340052303500523036005230340052387F
:10A0FE00370000000000600ABB36F909A60A2A0ADA
:10A10E00080A1C0A000000001B1B211752393920B7
:10A11E00484F4D45205A204F4E20535441525455CE
:10A12E00500D0A0052393920484F4D452059204FC5
:10A13E004E20535441525455500D0A005239392075
:10A14E00484F4D452058204F4E20535441525455A0
:10A15E00500D0A005239392041524455494E4F2074
:10A16E005354415254555020434F4D504C45544535
:10A17E000D0A002A004730004730300047310047B3
:10A18E00303100473238004630390046390046310A
:10A19E00310046313200463133004631340046310B
:10A1AE0035004631360046323000463231004632F6
:10A1BE0032004633310046333200463431004634E5
:10A1CE0032004634330046343400463631004638C9
:10A1DE003100463832004638330046383400200A03
:10A1EE000D005239392068616E646C6572203D3DF8
:10A1FE00204E554C4C0D0A005239390020726573B1
:10A20E00657474696E67206469676974616C207027
:10A21E00696E0020726573657474696E6720616E75
:10A22E00616C6F672070696E005239392045727209
:10A23E006F723A20696E76616C696420706172612A
:10A24E006D657465722069640D0A002051005238E4
:10A25E003100205841002058420020594100205919
:10A26E004200205A4100205A4200523832005239E0
:10A27E00392057696C6C207A65726F2058005239FC
:10A28E00392057696C6C207A65726F2059005239EB
:10A29E00392057696C6C207A65726F205A005238DB
:10A2AE0033200052323000686F6D650D0A00207346
:10A2BE007461200020637572200020656E6420009A
:10A2CE002068616C662000206C656E2000206D6930
:10A2DE006E2000206D617820002073706420005283
:10A2EE003231005000560052393920656D65726763
:10A2FE00656E63792073746F700D0A0052393920C0
:10A30E006572726F720D0A005239392073746F7054
:10A31E007065640D0A00523939206572726F7220B1
:10A32E00002064656163746976617465206D6F7475
:10A33E006F7220582064756520746F206D69737379
:10A34E00656420737465707300206465616374695D
:10A35E0076617465206D6F746F7220592064756517
:10A36E0020746F206D6973736564207374657073E8
:10A37E00002064656163746976617465206D6F7425
:10A38E006F72205A2064756520746F206D69737327
:10A39E006564207374657073005239392074696D69
:10A3AE00656F7574205820617869730D0A005239F3
:10A3BE00392074696D656F757420592061786973E1
:10A3CE000D0A005239392074696D656F7574205A03
:10A3DE0020617869730D0A005234310052393920E8
:10A3EE0043616C6962726174696F6E206572726F1F
:10A3FE00723A20696E76616C6964206178697320A7
:10A40E0073656C65637465640D0A00206178697309
:10A41E002000206174207374617274696E672070FD
:10A42E006F696E7400523233002063616C69627220
:10A43E006174696E67206C656E6774680020737452
:10A44E00657020636F756E743A2000523939206D35
:10A45E006F76656D656E7420646F6E650D0A0020F3
:10A46E00617420656E6420706F696E7400523939A4
:10A47E002043616C6962726174696F6E20657272DD
:10A48E006F723A20656E642073746F70206163740E
:10A49E00697665206265666F726520737461727489
:10A4AE000D0A00206D6F766520746F2073746172D3
:10A4BE007420666F722063616C6962726174696F79
:0EA4CE006E006E616E00696E66006F7666004D
:020000023000CC
:10E000000D9489F10D94B2F10D94B2F10D94B2F129
:10E010000D94B2F10D94B2F10D94B2F10D94B2F1F0
:10E020000D94B2F10D94B2F10D94B2F10D94B2F1E0
:10E030000D94B2F10D94B2F10D94B2F10D94B2F1D0
:10E040000D94B2F10D94B2F10D94B2F10D94B2F1C0
:10E050000D94B2F10D94B2F10D94B2F10D94B2F1B0
:10E060000D94B2F10D94B2F10D94B2F10D94B2F1A0
:10E070000D94B2F10D94B2F10D94B2F10D94B2F190
:10E080000D94B2F10D94B2F10D94B2F10D94B2F180
:10E090000D94B2F10D94B2F10D94B2F10D94B2F170
:10E0A0000D94B2F10D94B2F10D94B2F10D94B2F160
:10E0B0000D94B2F10D94B2F10D94B2F10D94B2F150
:10E0C0000D94B2F10D94B2F10D94B2F10D94B2F140
:10E0D0000D94B2F10D94B2F10D94B2F10D94B2F130
:10E0E0000D94B2F141546D656761323536300041AF
:10E0F000726475696E6F206578706C6F72657220DE
:10E1000073746B3530305632206279204D4C530099
:10E11000426F6F746C6F616465723E004875683F52
:10E1200000436F6D70696C6564206F6E203D200048
:10E130004350552054797065202020203D20005FF9
:10E140005F4156525F415243485F5F3D2000415658
:10E1500052204C696243205665723D20004743437C
:10E160002056657273696F6E203D20004350552024
:10E1700049442020202020203D20004C6F7720663D
:10E18000757365202020203D20004869676820665F
:10E190007573652020203D200045787420667573D6
:10E1A00065202020203D20004C6F636B2066757336
:10E1B000652020203D20004D617220203720323024
:10E1C000313300312E362E3800342E332E350056A2
:10E1D00023202020414444522020206F7020636F70
:10E1E00064652020202020696E73747275637469E1
:10E1F0006F6E2061646472202020496E74657272B3
:10E20000757074006E6F20766563746F7200726A49
:10E210006D702020006A6D70200057686174207056
:10E220006F72743A00506F7274206E6F7420737541
:10E2300070706F72746564004D7573742062652030
:10E2400061206C6574746572002000577269747483
:10E25000696E672045450052656164696E672045B7
:10E26000450045452065727220636E743D00504F35
:10E27000525400303D5A65726F2061646472003FF1
:10E280003D43505520737461747300403D454550C3
:10E29000524F4D207465737400423D426C696E6B41
:10E2A000204C454400453D44756D70204545505215
:10E2B0004F4D00463D44756D7020464C415348001B
:10E2C000483D48656C70004C3D4C69737420492F83
:10E2D0004F20506F72747300513D51756974005234
:10E2E0003D44756D702052414D00563D73686F7707
:10E2F00020696E7465727275707420566563746FF0
:10E30000727300593D506F727420626C696E6B00BD
:10E310002A0011241FBECFEFD1E2DEBFCDBF01E046
:10E320000CBF12E0A0E0B2E0EEE1FDEF03E00BBFB6
:10E3300002C007900D92A030B107D9F712E0A0E01B
:10E34000B2E001C01D92AE30B107E1F70F9460F367
:10E350000D948DFE01E20EBF0FEF0DBF11241FBE05
:10E360000D9460F30D9400F020E030E040ED57E0B4
:10E3700005C0FA013197F1F72F5F3F4F2817390792
:10E38000C0F308959C01260F311DC901A0E0B0E043
:10E390002F5F3F4FABBFFC018791882361F08093D3
:10E3A000C6008091C00086FFFCCF8091C0008064D1
:10E3B0008093C000EACF08958DE08093C6008091DD
:10E3C000C00086FFFCCF8091C00080648093C000B5
:10E3D0008AE08093C6008091C00086FFFCCF8091C8
:10E3E000C00080648093C00008950F94C2F10F9420
:10E3F000DCF10895FC019081992359F09093C600B7
:10E400008091C00086FFFCCF8091C0008064809323
:10E41000C0003196992379F70895282F982F929567
:10E420009F70892F805D8A3308F0895F8093C600D2
:10E430008091C00086FFFCCF8091C00080648093F3
:10E44000C000822F8F70982F905D9A3308F0995FEB
:10E450009093C6008091C00086FFFCCF8091C000E1
:10E4600080648093C00008959C01FB01853691056E
:10E470001CF46330710594F0C90164E670E00F94F8
:10E480002EFE605D7F4F6093C6008091C00086FFC6
:10E49000FCCF8091C00080648093C0002B30310598
:10E4A00014F43297B4F0C90164E670E00F942EFEC4
:10E4B0006AE070E00F942EFE605D7F4F6093C600AF
:10E4C0008091C00086FFFCCF8091C0008064809363
:10E4D000C000C9016AE070E00F942EFEC0968093E0
:10E4E000C6008091C00086FFFCCF8091C000806490
:10E4F0008093C00008951F93182F8EE692EE60E07F
:10E500000F94C2F11093C6008091C00086FFFCCF2B
:10E510008091C00080648093C0000F94DCF11F9153
:10E5200008952F923F924F925F926F927F928F92B7
:10E530009F92AF92BF92CF92DF92EF92FF920F9392
:10E540001F93DF93CF93CDB7DEB762970FB6F894E2
:10E55000DEBF0FBECDBF382E622ECA01DB015C01CB
:10E560006D01772420E2222E2E010894411C511CBB
:10E570008BC081E0A81680E0B80681E0C80680E084
:10E58000D80628F0C601AA27BB270F940DF2BB2797
:10E59000AD2D9C2D8B2D0F940DF28A2D0F940DF225
:10E5A0002092C6008091C00086FFFCCF8091C00001
:10E5B00080648093C0009DE29093C6008091C0006B
:10E5C00086FFFCCF8091C00080648093C0002092C1
:10E5D000C6008091C00086FFFCCF8091C00080649F
:10E5E0008093C00019828601750188249924A1E0D6
:10E5F0003A1651F03A1620F0B2E03B1661F409C029
:10E600000BBFF701779007C0C7010F9477FE782EF4
:10E6100002C0F7017080872D0F940DF22092C60082
:10E620008091C00086FFFCCF8091C0008064809301
:10E63000C000872D8052F401EF70F0708F3520F408
:10E64000E40DF51D708204C0E40DF51D8EE280839B
:10E650000894E11CF11C011D111D0894811C911CE2
:10E6600090E18916910409F0C2CF80E190E0A0E02A
:10E67000B0E0A80EB91ECA1EDB1E198AC2010F9493
:10E68000FAF10F94DCF16A94662009F072CF629679
:10E690000FB6F894DEBF0FBECDBFCF91DF911F91B3
:10E6A0000F91FF90EF90DF90CF90BF90AF909F9031
:10E6B0008F907F906F905F904F903F902F90089534
:10E6C0002F923F924F925F926F927F928F929F9282
:10E6D000AF92BF92CF92DF92EF92FF920F931F9370
:10E6E000DF93CF93CDB7DEB7CD53D1400FB6F894BB
:10E6F000DEBF0FBECDBF01E20EBF0FEF0DBF94B75F
:10E70000F894A89514BE80916000886180936000A1
:10E7100010926000789493FF05C0E0910002F091A0
:10E7200001021995279A2F9A8091C00082608093E8
:10E73000C00080E18093C40088E18093C1000000A4
:10E74000EE24FF24870144E0A42EB12CCC24DD2448
:10E7500024C0C5010197F1F70894E11CF11C011DCB
:10E76000111D21E2E2162EE4F20620E0020720E06D
:10E77000120718F031E0C32ED12CC801B70127ECE5
:10E780003BE140E050E00F9441FE611571058105C9
:10E79000910519F485B1805885B98091C00087FD35
:10E7A00003C0C114D104A9F2A6014F5F5F4FC25E3E
:10E7B000DE4F59834883CE51D140C25EDE4F8881FF
:10E7C0009981CE51D140019711F00D9410FEC05D9A
:10E7D000DE4F19821882C053D14060E0C15DDE4F28
:10E7E0001882CF52D14088249924C35DDE4F19820C
:10E7F0001882CD52D140C05EDE4F188219821A8233
:10E800001B82C052D140CE5CDE4F188219821A8220
:10E810001B82C253D140EE24FF2487010BBFF701B6
:10E8200007911691C45CDE4F19830883CC53D14005
:10E830000D940BFEC25EDE4F28813981CE51D1404E
:10E840002130310509F52091C600C25EDE4F1982E4
:10E850001882CE51D14022C02F5F3F4F4F4F5F4FA4
:10E86000213082E138078AE7480780E0580780F0C6
:10E87000C45CDE4FE881F981CC53D140EF5FFF4F9C
:10E8800019F0EE27FF27099420E030E040E050E047
:10E890008091C00087FFE0CF2091C600C35DDE4FAE
:10E8A00048815981CD52D1404F5F5F4FC35DDE4FEC
:10E8B00059834883CD52D140213209F063C64A3092
:10E8C000510508F05FC60894811C911C53E0851621
:10E8D000910409F059C600E010E018C081E280936D
:10E8E000C6008091C00086FFFCCF8091C00080648C
:10E8F0008093C0002F5F3F4F2931310579F70F9486
:10E90000DCF10F5F1F4F0530110519F020E030E0FA
:10E91000E5CF10920A0210920B0210920C02109294
:10E920000D02109206021092070210920802109235
:10E930000902109202021092030210920402109235
:10E9400005028FEE90EE60E00F94F5F180E191EE1C
:10E9500060E00F94C2F18091C00087FFFCCF9091DE
:10E96000C600903608F09F759032B8F09093C600BC
:10E970008091C00086FFFCCF8091C00080648093AE
:10E98000C000A0E2A093C6008091C00086FFFCCF2B
:10E990008091C00080648093C000983409F4D7C18E
:10E9A0009934B8F4923409F459C1933458F490333B
:10E9B00019F1903308F4E3C59F33A1F1903409F0C5
:10E9C000DEC5BDC0953409F470C1963409F0D7C5D1
:10E9D00098C1923509F42BC2933538F49C3409F46C
:10E9E000F5C1913509F0CBC518C2963509F445C279
:10E9F000993509F0C4C567C483E792EE62E00F94CD
:10EA0000F5F110920602109207021092080210927D
:10EA1000090210920A0210920B0210920C0210923C
:10EA20000D0213C18FE792EE62E00F94F5F18FEEC5
:10EA300090EE60E00F94F5F181E291EE60E00F94CA
:10EA4000C2F187EB91EE60E00F94F5F180E391EE77
:10EA500060E00F94C2F184EE90EE60E00F94F5F167
:10EA60008FE391EE60E00F94C2F186E090E061E008
:10EA700070E00F9434F20F94DCF18DE591EE60E0DC
:10EA80000F94C2F189EC91EE60E00F94F5F18EE401
:10EA900091EE60E00F94C2F183EC91EE60E00F9490
:10EAA000F5F18CE691EE60E00F94C2F18EE10F94E7
:10EAB0000DF288E90F940DF281E00F940DF20F949E
:10EAC000DCF18BE791EE60E00F94C2F119E0E0E039
:10EAD000F0E010935700E4918E2F0F940DF20F94F5
:10EAE000DCF18AE891EE60E00F94C2F1E3E0F0E03F
:10EAF00010935700E4918E2F0F940DF20F94DCF1D8
:10EB000089E991EE60E00F94C2F1E2E0F0E0109349
:10EB10005700E4918E2F0F940DF20F94DCF188EAE8
:10EB200091EE60E00F94C2F1E1E0F0E01093570045
:10EB30001491812F0F940DF20F94DCF107CF8BE825
:10EB400092EE62E00F94F5F18BE492EE60E00F94A8
:10EB5000F5F10F94DCF100E010E019C0C8016F2D51
:10EB60000F947FFEFF2031F489E492EE60E00F9471
:10EB7000C2F10BC0F092C6008091C00086FFFCCFAE
:10EB80008091C00080648093C0000F5F1F4FC80158
:10EB900081519F41A0E0B0E0ABBFFC01F790BAE229
:10EBA000FB1621F0E2E000301E07C1F60F94DCF105
:10EBB0000F94DCF187E592EE60E00F94F5F10F948D
:10EBC000DCF1CC24DD2400E010E01EC0C8010F946D
:10EBD00077FEF82E882331F489E492EE60E00F94FA
:10EBE000C2F10BC08093C6008091C00086FFFCCFAD
:10EBF0008091C00080648093C000FE1419F00894D6
:10EC0000C11CD11C0F5F1F4FC80181519F41A0E063
:10EC1000B0E0ABBFFC01E790FAE2EF1621F022E092
:10EC20000030120799F60F94DCF10F94DCF182E6C4
:10EC300092EE60E00F94C2F1C60161E070E00F94C3
:10EC400034F20F94DCF10F94DCF110920202109276
:10EC50000302109204021092050278CE89E992EE26
:10EC600062E00F94F5F1279A2F9A16C02F9880E052
:10EC700090E0E0EDF7E03197F1F7019684369105E9
:10EC8000C1F72F9A80E090E0E0EDF7E03197F1F7DF
:10EC9000019684369105C1F78091C00087FFE6CFC9
:10ECA0008091C00087FFFCCF64C485EA92EE62E0E9
:10ECB0000F94F5F140910202509103026091040219
:10ECC0007091050281E020E10F9491F2809102029F
:10ECD00090910302A0910402B091050280509F4FD1
:10ECE000AF4FBF4F8093020290930302A0930402A0
:10ECF000B093050280509041A040B04008F426CE69
:10ED0000A4CF83EB92EE62E00F94F5F140910602FE
:10ED100050910702609108027091090280E020E1A1
:10ED20000F9491F28091060290910702A09108023F
:10ED3000B091090280509F4FAF4FBF4F80930602A2
:10ED400090930702A0930802B0930902FFCD80ECD4
:10ED500092EE62E00F94F5F183E792EE60E00F949B
:10ED6000F5F18FE792EE60E00F94F5F18BE892EE0B
:10ED700060E00F94F5F189E992EE60E00F94F5F10F
:10ED800085EA92EE60E00F94F5F183EB92EE60E09D
:10ED90000F94F5F180EC92EE60E00F94F5F187ECC2
:10EDA00092EE60E00F94F5F188ED92EE60E00F9442
:10EDB000F5F18FED92EE60E00F94F5F18AEE92EEB0
:10EDC00060E00F94F5F183E093EEBDCD87EC92EE19
:10EDD00062E00F94F5F181E40F947BF282E40F94EA
:10EDE0007BF283E40F947BF284E40F947BF285E45E
:10EDF0000F947BF286E40F947BF287E40F947BF20E
:10EE000088E40F947BF28AE40F947BF28BE40F94F6
:10EE10007BF28CE40F947BF299CD88ED92EE62E068
:10EE20000F94F5F1772473948824992409C48FED05
:10EE300092EE62E00F94F5F140910A0250910B02BC
:10EE400060910C0270910D0282E020E10F9491F22A
:10EE500080910A0290910B02A0910C02B0910D02D8
:10EE600080509F4FAF4FBF4F80930A0290930B0289
:10EE7000A0930C02B0930D0269CD8AEE92EE62E08F
:10EE80000F94F5F184EE90EE60E00F94F5F18FECC5
:10EE900091EE60E00F94F5F1662477244301CC5D98
:10EEA000DE4F19821882C452D140D401C301B695F5
:10EEB000A79597958795CA5DDE4F88839983AA8326
:10EEC000BB83C652D140CC5DDE4FA881B981C4520C
:10EED000D1401196CC5DDE4FB983A883C452D14096
:10EEE000CD0162E070E00F9434F2B0E2B093C6005E
:10EEF0008091C00086FFFCCF8091C0008064809329
:10EF0000C000EDE2E093C6008091C00086FFFCCF18
:10EF10008091C00080648093C000F0E2F093C6004E
:10EF20008091C00086FFFCCF8091C00080648093F8
:10EF3000C000CA5DDE4FE880F9800A811B81C6529D
:10EF4000D140BB27A12F902F8F2D0F940DF2CA5DBA
:10EF5000DE4F8881C652D1400F940DF2B0E2FB2EF5
:10EF6000F092C6008091C00086FFFCCF8091C00067
:10EF700080648093C0000DE30093C6008091C000C0
:10EF800086FFFCCF8091C00080648093C00010E2B7
:10EF90001093C6008091C00086FFFCCF8091C00016
:10EFA00080648093C0008BBEF3012791C65DDE4F65
:10EFB0002883CA52D140A22EBB24CC24DD2408943D
:10EFC000611C711C811C911C8BBEF3018791282E42
:10EFD0003324442455240894611C711C811C911C09
:10EFE0008BBEF3013791C55DDE4F3883CB52D140E4
:10EFF0000894611C711C811C911C8BBEF30147910C
:10F00000C45DDE4F4883CC52D140ADEFEA2EAFEF66
:10F01000FA2EAFEF0A2FAFEF1A2F6E0C7F1C801E57
:10F02000911E142D032DF22CEE24EA0CFB1C0C1D5A
:10F030001D1D0F940DF220E22093C6008091C000A8
:10F0400086FFFCCF8091C00080648093C000C65DC5
:10F05000DE4F8881CA52D1400F940DF230E23093D6
:10F06000C6008091C00086FFFCCF8091C000806404
:10F070008093C000C45DDE4F8881CC52D1400F9494
:10F080000DF240E24093C6008091C00086FFFCCFA5
:10F090008091C00080648093C000C55DDE4F888190
:10F0A000CB52D1400F940DF250E25093C6008091A4
:10F0B000C00086FFFCCF8091C00080648093C000B8
:10F0C0008FEFE8168FEFF80680E0080780E018075A
:10F0D00031F484E092EE60E00F94C2F1DFC0D80119
:10F0E000C7018070907CA070B0708050904CA040A0
:10F0F000B040D1F52FEF3FE340E050E0E222F322B1
:10F1000004231523CA5DDE4FA880B980CA80DB8046
:10F11000C652D140AE0CBF1CC01ED11EAA0CBB1CD7
:10F12000CC1CDD1C8EE092EE60E00F94C2F1BB2798
:10F13000A12F902F8F2D0F940DF28E2D0F940DF285
:10F1400030E23093C6008091C00086FFFCCF8091F2
:10F15000C00080648093C0004EE34093C60080915D
:10F16000C00086FFFCCF87C08EE09EEFA0E0B0E03D
:10F17000E822F9220A231B239CE0E91694E9F90608
:10F1800090E0090790E0190709F088C0C45DDE4FE0
:10F19000A881CC52D140EA2EFF2400E010E0102FCD
:10F1A0000F2DFE2CEE24C55DDE4FB881CB52D14031
:10F1B000EB0EF11C011D111DD601C501817090706F
:10F1C000A070B070DC0199278827E80EF91E0A1F8D
:10F1D0001B1F20EF30E040E050E0A222B322C42207
:10F1E000D52241E1AA0CBB1CCC1CDD1C4A95D1F7F1
:10F1F000EA0CFB1C0C1D1D1D81E090E0A0E0B0E0BE
:10F20000282239224A225B2235E1220C331C441C7D
:10F21000551C3A95D1F7E20CF31C041D151D57013E
:10F220006801AA0CBB1CCC1CDD1C85E192EE60E0E1
:10F230000F94C2F1C801AA27BB270F940DF2BB2778
:10F24000A12F902F8F2D0F940DF28E2D0F940DF274
:10F2500090E29093C6008091C00086FFFCCF809121
:10F26000C00080648093C000AEE3A093C60080918C
:10F27000C00086FFFCCF8091C00080648093C000F6
:10F28000C601AA27BB270F940DF2BB27AD2D9C2DDD
:10F290008B2D0F940DF28A2D0F940DF20F94DCF14B
:10F2A000CC5DDE4FE881F981C452D140F99709F471
:10F2B0004DCBF4E0EF2EF12C012D112D6E0C7F1CA7
:10F2C000801E911EF2CD83E093EE62E00F94F5F183
:10F2D0008AE192EE60E00F94C2F18091C00087FF56
:10F2E000FCCF1091C6001F751093C6008091C0001E
:10F2F00086FFFCCF8091C00080648093C0000F9493
:10F30000DCF1812F81548A3108F036C1163409F4BA
:10F3100095C0173490F4133409F44EC0143430F40B
:10F320001134F1F0123409F01DC130C0143409F465
:10F3300059C0153409F016C16BC01A3409F4C4C0A1
:10F340001B3438F4173409F48FC0183409F00AC19B
:10F35000A1C01B3409F4D2C01C3409F003C1E8C0B9
:10F360008FEF81B90DC082B1809582B980E090E0C5
:10F37000E0EDF7E03197F1F70196883C9105C1F790
:10F380008091C00087FFEFCF12B8EFC08FEF84B934
:10F390000DC085B1809585B980E090E0E0EDF7E0A3
:10F3A0003197F1F70196883C9105C1F78091C00033
:10F3B00087FFEFCF15B8D9C08FEF87B90DC088B1DF
:10F3C000809588B980E090E0E0EDF7E03197F1F7C3
:10F3D0000196883C9105C1F78091C00087FFEFCF6F
:10F3E00018B8C3C08FEF8AB90DC08BB180958BB9A7
:10F3F00080E090E0E0EDF7E03197F1F70196883C8E
:10F400009105C1F78091C00087FFEFCF1BB8ADC059
:10F410008FEF8DB90DC08EB180958EB980E090E0F0
:10F42000E0EDF7E03197F1F70196883C9105C1F7DF
:10F430008091C00087FFEFCF1EB897C08FEF80BBD1
:10F440000DC081B3809581BB80E090E0E0EDF7E0F6
:10F450003197F1F70196883C9105C1F78091C00082
:10F4600087FFEFCF11BA81C08FEF83BB0DC084B38C
:10F47000809584BB80E090E0E0EDF7E03197F1F714
:10F480000196883C9105C1F78091C00087FFEFCFBE
:10F4900014BA6BC08FEF809301010FC080910201FD
:10F4A00080958093020180E090E0E0EDF7E03197F5
:10F4B000F1F70196883C9105C1F78091C00087FF64
:10F4C000EDCF1092020151C08FEF809304010FC065
:10F4D0008091050180958093050180E090E0E0ED4A
:10F4E000F7E03197F1F70196883C9105C1F78091DB
:10F4F000C00087FFEDCF1092050137C08FEF8093DA
:10F5000007010FC08091080180958093080180E079
:10F5100090E0E0EDF7E03197F1F70196883C910536
:10F52000C1F78091C00087FFEDCF109208011DC088
:10F530008FEF80930A010FC080910B01809580931B
:10F540000B0180E090E0E0EDF7E03197F1F70196F4
:10F55000883C9105C1F78091C00087FFEDCF1092E4
:10F560000B0103C085E292EEEEC98091C00087FFD7
:10F57000FCCF8091C600EAC988E392EEE4C98CE131
:10F5800091EEE1C988249924933011F1943028F444
:10F59000913089F09230B8F408C0953061F195301F
:10F5A000F0F0963009F048C043C02B3109F042C951
:10F5B00091E06BE13FC96227C15DDE4F2883CF52E6
:10F5C000D14092E037C9B22FA0E0622793E032C960
:10F5D000822F90E0A82BB92B622794E02BC92E3004
:10F5E00009F039C3622795E0C05DDE4F19821882A9
:10F5F000C053D1401FC9E1E0F0E0EC0FFD1FC05D3A
:10F60000DE4F08811981C053D140E00FF11F2083E4
:10F610000F5F1F4FC05DDE4F19830883C053D14079
:10F6200062270A171B0709F005C9D80196E002C92D
:10F63000261709F010C303C0973009F0FBC87724E0
:10F640009981933109F412C19431C8F4963009F4C8
:10F65000D8C0973050F4923009F406C1933009F4C1
:10F660006DC0913009F059C253C0913109F477C08F
:10F67000923108F0BBC0903109F04FC2F5C098310B
:10F6800009F487C0993150F4953109F4EFC09531F0
:10F6900008F4C6C1963109F040C2C2C19A3109F4DA
:10F6A0006CC09A3108F491C09B3109F45BC09D3164
:10F6B00009F033C29D81903359F48F81882311F46E
:10F6C0009EE11CC0813011F091E018C098E916C08D
:10F6D000892F807591F0903539F4E0E0F0E089E011
:10F6E0008093570094910AC0983539F4E3E0F0E034
:10F6F00089E080935700949101C090E01A821B82A8
:10F700008D818C831D829E831F8227E030E009C299
:10F710001A8288E08B8381E48C8386E58D8382E581
:10F720008E8389E48F8383E5888780E589878FE5E9
:10F730008A8782E38B872BE030E0F3C18A818139AD
:10F7400041F0823941F0803911F48FE005C080E04A
:10F7500003C082E001C08AE01A828B8344C0772410
:10F76000739482C08D81882311F48EE12CC0813086
:10F7700011F081E028C088E926C01A82E1E0F0E0BB
:10F7800089E08093570084918B831C8224E030E0D1
:10F79000C8C18B81803589F48C81883039F4E2E0EE
:10F7A000F0E089E08093570084910DC0E0E0F0E044
:10F7B00089E080935700849106C0E3E0F0E089E09F
:10F7C0008093570084911A82DFCF8D81836C99E0FA
:10F7D000E1E0F0E0082E90935700E89507B600FCB2
:10F7E000FDCF1A821B8223E030E09BC180EC8A832C
:10F7F000CE5CDE4F188219821A821B82C253D1401E
:10F800008EC18A8190E0A0E0B0E0582F44273327D2
:10F8100022278B8190E0A0E0B0E0DC0199278827C7
:10F82000282B392B4A2B5B2B8D8190E0A0E0B0E098
:10F83000282B392B4A2B5B2B8C8190E0A0E0B0E089
:10F84000BA2FA92F982F8827282B392B4A2B5B2BCF
:10F85000220F331F441F551FC05EDE4F288339839C
:10F860004A835B83C052D1401A8259C13A81C95C34
:10F87000DE4F3883C753D140CA5CDE4F1882C6536F
:10F88000D1408B81C82EDD24CA5CDE4F488159816E
:10F89000C653D140C42AD52A933109F082C0CE5C28
:10F8A000DE4F88819981AA81BB81C253D1408050AB
:10F8B000904CA340B04030F583E0CE5CDE4FE88052
:10F8C000F9800A811B81C253D140F70100935B008C
:10F8D00080935700E89507B600FCFDCFCE5CDE4F65
:10F8E000088119812A813B81C253D14000501F4FAA
:10F8F0002F4F3F4FCE5CDE4F088319832A833B8313
:10F90000C253D140C05EDE4F488159816A817B81FC
:10F91000C052D140DE011B9631E08C9111962C91A2
:10F9200011971296C75CDE4F2883C953D140C85C3B
:10F93000DE4F1882C853D14090E0C85CDE4FE881AA
:10F94000F981C853D1408E2B9F2B0C01FA01609393
:10F950005B0030935700E89511244E5F5F4F6F4F67
:10F960007F4F0EEFE02E0FEFF02ECE0CDF1CC114F8
:10F97000D10499F685E0C05EDE4F088119812A81A5
:10F980003B81C052D140F80120935B008093570027
:10F99000E89507B600FCFDCF81E180935700E8951C
:10F9A00035C0C05EDE4F88819981AA81BB81C0527B
:10F9B000D140B695A795979587957C018601ABE0D8
:10F9C000AA2EB12CAC0EBD1E0BC0D5016D915D01F0
:10F9D000C7010F947FFE0894E11CF11C01501040F8
:10F9E0000115110591F7A60160E070E0440F551F65
:10F9F000661F771FC05EDE4FE880F9800A811B8199
:10FA0000C052D1404E0D5F1D601F711F1A82C05E33
:10FA1000DE4F488359836A837B83C052D1407FC0C5
:10FA2000FA80C55CDE4FF882CB53D140C65CDE4F16
:10FA30001882CA53D1408B81C82EDD24C65CDE4FAC
:10FA400008811981CA53D140C02AD12A1A828981DA
:10FA5000BE016D5F7F4F843121F59601C05EDE4FA0
:10FA6000E880F9800A811B81C052D1400BBFF701A9
:10FA700087919691DB018C9311969C936E5F7F4FDB
:10FA8000D801C7010296A11DB11DC05EDE4F88835B
:10FA90009983AA83BB83C052D14022503040F1F6F3
:10FAA00036C0C05EDE4F288139814A815B81C052F9
:10FAB000D1400894C108D108760100E010E0089414
:10FAC000C11CD11C0894E11CF11C011D111DE20E8A
:10FAD000F31E041F151F21BDBB27A52F942F832FB5
:10FAE00082BD2F5F3F4F4F4F5F4FF89A80B5DB01CC
:10FAF0008D93BD012E153F054007510761F7C05E8C
:10FB0000DE4F288339834A835B83C052D1409601FC
:10FB10002D5F3F4FFB01108204C080EC8A8322E0FE
:10FB200030E08BE18093C6008091C00086FFFCCF5F
:10FB30008091C00080648093C000C15DDE4FF88179
:10FB4000CF52D140F093C6008091C00086FFFCCF19
:10FB50008091C00080648093C000432F3093C60022
:10FB60008091C00086FFFCCF8091C00080648093AC
:10FB7000C000922F2093C6008091C00086FFFCCF6A
:10FB80008091C00080648093C0008EE08093C600A6
:10FB90008091C00086FFFCCF8091C000806480937C
:10FBA000C00065E1C15DDE4FE880CF52D1406E25D7
:10FBB00069276427FE01319610C090819093C6009A
:10FBC0008091C00086FFFCCF31968091C000806498
:10FBD0008093C0006927215030402115310569F715
:10FBE0006093C6008091C00086FFFCCF8091C0006A
:10FBF00080648093C00085B1805885B9772081F4F6
:10FC0000C15DDE4F0881CF52D1400F5FC15DDE4F35
:10FC10000883CF52D14090E0A0E0B0E00D941AF4F8
:10FC200027982F9880E090E020ED37E0F901319798
:10FC3000F1F7019684369105C9F700008091C00064
:10FC40008D7F8093C00081E180935700E895EE2777
:10FC5000FF270994FFCF90E00D941AF497FB092E2B
:10FC600007260AD077FD04D02ED006D000201AF443
:10FC7000709561957F4F0895F6F7909581959F4F08
:10FC80000895A1E21A2EAA1BBB1BFD010DC0AA1FDD
:10FC9000BB1FEE1FFF1FA217B307E407F50720F0F5
:10FCA000A21BB30BE40BF50B661F771F881F991F70
:10FCB0001A9469F760957095809590959B01AC01B9
:10FCC000BD01CF010895AA1BBB1B51E107C0AA1FAC
:10FCD000BB1FA617B70710F0A61BB70B881F991FED
:10FCE0005A95A9F780959095BC01CD010895F99991
:10FCF000FECF92BD81BDF89A992780B50895262F31
:10FD0000F999FECF1FBA92BD81BD20BD0FB6F89400
:0EFD1000FA9AF99A0FBE01960895F894FFCF63
:040000033000E000E9
:00000001FF
